:020000040800F2
:1000000000070020F1020008E133000899330008DE
:10001000C133000899330008B9330008F30200081F
:10002000F3020008F3020008F3020008CD430008C1
:10003000F3020008F3020008F3020008F3020008CC
:10004000F3020008F3020008F3020008F3020008BC
:10005000F3020008F302000881640008AD640008A0
:10006000D96400080565000831650008914400085E
:10007000B9440008E5440008114500083D45000862
:100080006545000891450008F3020008493300085F
:10009000713300085D330008853300085D65000892
:1000A000F3020008F3020008F3020008F30200085C
:1000B000F3020008F3020008F3020008F30200084C
:1000C000F3020008F3020008F3020008F30200083C
:1000D000F302000835660008F3020008F302000886
:1000E000C1650008F3020008F3020008F3020008EB
:1000F000F3020008F3020008F3020008BD450008FF
:10010000F3020008F30200085D660008F30200082D
:10011000F3020008F3020008F3020008F3020008EB
:10012000E9450008114600083D46000869460008F8
:1001300095460008F3020008F3020008F3020008E5
:10014000F3020008F3020008F3020008F3020008BB
:10015000BD460008E946000815470008F3020008FC
:10016000F3020008F3020008F3020008F30200089B
:10017000F3020008F3020008F3020008F30200088B
:10018000F3020008F3020008F302000849660008C1
:10019000F3020008F3020008F3020008F30200086B
:1001A000F3020008F3020008F3020008F30200085B
:1001B000F3020008F3020008F3020008F30200084B
:1001C000F3020008F3020008F3020008F30200083B
:1001D000F3020008F3020008F3020008F30200082B
:1001E000F3020008F3020008F3020008F30200081B
:1001F000F3020008F3020008F3020008F30200080B
:10020000F3020008F3020008F3020008F3020008FA
:10021000F3020008F3020008F3020008F3020008EA
:10022000F3020008F3020008F3020008F3020008DA
:10023000F3020008F3020008F3020008F3020008CA
:10024000F3020008F3020008F3020008F3020008BA
:10025000F3020008F3020008F3020008F3020008AA
:10026000F3020008F3020008F3020008F30200089A
:10027000F3020008F3020008F3020008F30200088A
:10028000F3020008F3020008F3020008F30200087A
:10029000F3020008F3020008F3020008F30200086A
:1002A000F3020008F3020008F3020008F30200085A
:1002B000F3020008F3020008F3020008F30200084A
:1002C000F3020008F3020008F3020008F30200083A
:1002D000F3020008F3020008F3020008F30200082A
:1002E000CD16000800000000000000000000000023
:1002F00002E000F000F8FEE772B6374880F30888A5
:10030000364880F3098836483649086040F20000D4
:10031000CCF200004EF63471CEF200010860BFF35B
:100320004F8FBFF36F8F40F20000C0F2F0004EF627
:100330008851CEF200010860BFF34F8FBFF36F8F7B
:100340004FF00000E1EE100A4EF63C71CEF20001D3
:100350000860062080F31488BFF36F8F05F020FC3F
:1003600005F05CFE4FF055301F491B4A91423CBFDF
:1003700041F8040BFAE71D49184A91423CBF41F885
:10038000040BFAE71A491B4A1B4B9A423EBF51F82D
:10039000040B42F8040BF8E700201849184A914270
:1003A0003CBF41F8040BFAE705F038FC05F0BCFE51
:1003B000144C154DAC4203DA54F8041B8847F9E796
:1003C00000F042F8114C124DAC4203DA54F8041B11
:1003D0008847F9E705F020BC000700200023002033
:1003E0000000000808ED00E00001002000070020E8
:1003F000786B0008002300203C23002040230020CD
:10040000E4700020E0020008E4020008E4020008B2
:10041000E40200082DE9F04F2DED108AC1F80CD050
:10042000D0F80CD0BDEC108ABDE8F08F002383F328
:1004300011882846A047002004F00CFFFEE704F0D6
:1004400091FE00DFFEE70000F8B501F055F901F07C
:1004500003FA01F04DFB05F0FFFA074605F096FBA5
:100460000546A8BB1F4B9F4232D001339F4232D07A
:1004700027F0FF021C4B9A4230D12E4642F21074F4
:10048000F8B200F06FFF00F073FF08B100242646B9
:1004900001F0BEFD20B10024032000F079F82646CB
:1004A00035B1124B9F4203D0002405F067FB26466E
:1004B000002005F0DBFA0EB100F080F801F0EAFA56
:1004C00000F08AFF204600F00BF900F077F8F9E71A
:1004D0002E460024D7E704460126D4E7064641F21B
:1004E0008834D0E7010007B0000008B0263A09B010
:1004F00008B501F07DF9A0F120035842584108BD2C
:1005000007B541F21203022101A8ADF8043001F051
:100510008DF903B05DF804FB38B5302383F31188FF
:10052000174803680BB104F053FF0023154A4FF43A
:100530007A71134804F042FF002383F31188124CB0
:10054000236813B12368013B2360636813B16368B8
:10055000013B63600D4D2B7833B963687BB9022092
:1005600001F02EFA322363602B78032B07D16368E6
:100570002BB9022001F024FA4FF47A73636038BD7E
:100580004023002019050008602400205823002083
:10059000084B187003280CD8DFE800F008050208A3
:1005A000022001F00BBA022001F006BA024B002231
:1005B0005A6070475823002060240020F8B501F0ED
:1005C00027FD30B13E4B03221A7000223D4B5A608A
:1005D000F8BD3D4B3D4A1C4619680131F8D0043343
:1005E0009342F9D162683A4B9A42F1D9394B9B68F0
:1005F00003F1006303F580239A42E9D205F092FAF1
:1006000005F0A4FA002001F04DF90220FFF7C0FF29
:10061000314B00219A6C99641A6F19671A6FDA6C62
:10062000D9645A6F59675A6F1A6D19659A6F99672D
:100630009B6F72B64FF0E023C3F8084DD4E9000475
:10064000BFF34F8FBFF36F8F244AC2F88410BFF3FC
:100650004F8F536923F480335361BFF34F8FD2F828
:10066000803043F6E076C3F3C905C3F34E335B0134
:1006700003EA060C29464CEA81770139C2F8747204
:10068000F9D2203B13F1200FF2D1BFF34F8FBFF30C
:100690006F8FBFF34F8FBFF36F8F536923F4003316
:1006A00053610023C2F85032BFF34F8FBFF36F8FF7
:1006B000302383F31188854680F30888204787E735
:1006C00058230020602400200000040820000408B3
:1006D000FFFF0308002300200045025800ED00E062
:1006E0002DE9F04F93B0B74B2022FF2100900AA8CC
:1006F0009D6801F079F9B44A1378A3B90121B34890
:1007000011700360302383F3118803680BB104F088
:100710005FFE0023AE4A4FF47A71AC4804F04EFEFF
:10072000002383F31188009B13B1AA4B009A1A602F
:10073000A94A1378032B03D000231370A54A5360F2
:100740004FF0000A009CD3465646D146012001F0E6
:1007500035F924B19F4B1B68002B00F02C82002040
:1007600001F046F80390039B002B01DA00F088FEAD
:10077000039B002BEDDB012001F01EF9039B213BC5
:100780001F2BE3D801A252F823F000BF0D08000888
:1007900035080008C90800084D0700084D07000883
:1007A0004D0700085B0900082B0B0008450A0008EC
:1007B000A70A0008CF0A0008F50A00084D0700083C
:1007C000070B00084D070008790B0008AD0800086A
:1007D0004D070008BD0B000819080008AD08000807
:1007E0004D070008A70A00084D0700084D0700083C
:1007F0004D0700084D0700084D0700084D07000889
:100800004D0700084D070008C90800080220FFF73F
:100810006FFE002840F0F981009B022105A8BAF183
:10082000000F08BF1C4641F21233ADF8143000F03F
:10083000FDFF8BE74FF47A7000F0DAFF071EEBDB69
:100840000220FFF755FE0028E6D0013F052F00F2F9
:10085000DE81DFE807F0030A0D10133605230421BB
:1008600005A8059300F0E2FF17E004215548F9E7D9
:1008700004215A48F6E704215948F3E74FF01C08D1
:10088000404608F1040801F00FF80421059005A87E
:1008900000F0CCFFB8F12C0FF2D101204FF000098D
:1008A00000FA07F747EA0B0B5FFA8BFB01F0E8F859
:1008B00026B10BF00B030B2B08BF0024FFF720FE23
:1008C00044E704214748CDE7002EA5D00BF00B03E9
:1008D0000B2BA1D10220FFF70BFE074600289BD06F
:1008E0000120002600F0DEFF0220FFF751FE1FFA74
:1008F00086F8404600F0E6FF0446B0B10399404652
:100900000136A1F140025142514100F0F3FF0028AD
:10091000EDD1BA46044641F21213022105A83E4623
:10092000ADF8143000F082FF10E725460120FFF7F4
:100930002FFE244B9B68AB4207D9284600F0B4FF3A
:10094000013040F067810435F3E70025224BBA46B9
:100950003E461D701F4B5D60A8E7002E3FF45CAF64
:100960000BF00B030B2B7FF457AF0220FFF710FEA9
:10097000322000F03DFFB0F10008FFF64DAF18F057
:1009800003077FF449AF0F4A08EB050392689342CF
:100990003FF642AFB8F5807F3FF73EAF124BB84508
:1009A000019323DD4FF47A7000F022FF0390039A45
:1009B000002AFFF631AF039A0137019B03F8012BA0
:1009C000EDE700BF002300205C240020402300202E
:1009D000190500086024002058230020042300206B
:1009E000082300200C2300205C230020C820FFF7F0
:1009F0007FFD074600283FF40FAF1F2D11D8C5F12A
:100A000020020AAB25F0030084494245184428BF60
:100A10004246019200F0D6FF019AFF217F4800F084
:100A2000E3FF4FEAA803C8F387027C4928460193F5
:100A300000F0E2FF064600283FF46DAF019B05EB96
:100A4000830533E70220FFF753FD00283FF4E4AEAF
:100A500000F062FF00283FF4DFAE0027B846704B7D
:100A60009B68BB4218D91F2F11D80A9B01330ED0A7
:100A700027F0030312AA134453F8203C0593404681
:100A8000042205A9043701F0ADFA8046E7E73846AD
:100A900000F00AFF0590F2E7CDF81480042105A8C4
:100AA00000F0C4FE02E70023642104A8049300F0D0
:100AB000B3FE00287FF4B0AE0220FFF719FD002836
:100AC0003FF4AAAE049800F01DFF0590E6E700236E
:100AD000642104A8049300F09FFE00287FF49CAEDC
:100AE0000220FFF705FD00283FF496AE049800F0C1
:100AF0000BFFEAE70220FFF7FBFC00283FF48CAE77
:100B000000F01AFFE1E70220FFF7F2FC00283FF4B3
:100B100083AE05A9142000F015FF074604210490B8
:100B200004A800F083FE3946B9E7322000F060FEE9
:100B3000071EFFF671AEBB077FF46EAE384A07EBB7
:100B40000903926893423FF667AE0220FFF7D0FC9C
:100B500000283FF461AE27F003074F44B9453FF446
:100B6000A5AE484609F1040900F09EFE0421059057
:100B700005A800F05BFEF1E74FF47A70FFF7B8FCD0
:100B800000283FF449AE00F0C7FE002844D00A9B7D
:100B900001330BD008220AA9002000F02DFF002805
:100BA0003AD02022FF210AA800F01EFFFFF7A8FC80
:100BB0001C4804F055FB13B0BDE8F08F002E3FF445
:100BC0002BAE0BF00B030B2B7FF426AE002364211E
:100BD00005A8059300F020FE074600287FF41CAE10
:100BE0000220FFF785FC804600283FF415AEFFF792
:100BF00087FC41F2883004F033FB059800F05EFF7B
:100C000046463C4600F03CFFA0E506464EE64FF067
:100C1000000901E6BA467EE637467CE65C23002002
:100C200000230020A0860100094A49F269001368E8
:100C300099B21B0C00FB013344F250611360054B69
:100C4000186882B2000C01FB0200186080B2704785
:100C500014230020102300200021102210B5044688
:100C600000F0C2FE034B03CB206061601868A060F7
:100C700010BD00BF00E8F11F2DE9F041ADF54E7D3C
:100C80000D46002140F275126CAC07460EA80D917E
:100C900000F0AAFE4FF4C4720021204600F0A4FE2A
:100CA0000DF1340802F0A4FB4FF47A72264BB0FB2E
:100CB000F2F0186093E80700022384E807000DF5BE
:100CC000E9702382FFF7C8FF41F204331F4907A8E8
:100CD000238405F04FFD15230DF2E3220DF12C0CBA
:100CE00084F8323107AB1E46083203CE664542F81F
:100CF000080C42F8041C3346F5D1306841461060B8
:100D0000204633791371012200F052FF002380B294
:100D1000E97E0393AB7E029305F11903019301234E
:100D2000009307A3D3E90023CDE90480384602F0FD
:100D30001DFF0DF54E7DBDE8F08100BFAFF30080D3
:100D40009E6AC421818A46EE6824002084670008D8
:100D50002DE9F0412C4CDAB080460D46237A5BBB7E
:100D600027A9284601F048F80746002842D19DF8F7
:100D70009D60C82E3ED801464FF4A662204600F082
:100D800033FE4FF4807332460DF19E01C4F8F83102
:100D90004FF4007304F109002644C4F80C334FF4F7
:100DA0004073C4F8203400F00DFE9DF89C3077723B
:100DB00023720BB9EB7E237206AC8122002127A897
:100DC00000F012FE0122214627A801F05BF8002363
:100DD00080B2E97E0393AB7E029305F11903019380
:100DE0002823CDE904400093404605A3D3E900231E
:100DF00002F0BCFE5AB0BDE8F08100BFAFF3008046
:100E000026417272DF25D7B7305E0020F0B5254E3F
:100E10004FF48A75F1B0002405FB006596F8D830D0
:100E2000D822214685F8DC303AA885F8E84006AF9C
:100E300000F0DAFD06F1090000F0CEFDD5F8E4304F
:100E4000C2B206F109018DF8F0000DF1F100CDE913
:100E50003A3400F0B7FD394601223AA801F048F8CB
:100E6000082380B2317ACDE9047001270E48CDE91C
:100E7000023706F1D80301933023009307A3D3E987
:100E8000002302F073FEA04206DD02F0B1FAC5F8BD
:100E9000E000384671B0F0BD2046FBE778F6339F9E
:100EA00093CACD8D305E0020803400202DE9F04FB4
:100EB000264F87B0DFF8A080254E384602F082FE2C
:100EC000034600283AD00024224DADF81440A14634
:100ED0000294A246CDE90344027B8DF8142003AAB4
:100EE0009968406803C21B6843F0004302932B6873
:100EF00004F5A664D3F810B002F07CFA10EB0802F7
:100F0000CDF800A0284605F5A65541F1000302A939
:100F1000D8470028C8BF49F00109B4F5266FE6D1CB
:100F2000B9F1000F05D0384602F050FE86F800A057
:100F3000C3E73378072B04D80133337007B0BDE81B
:100F4000F08F024802F042FEF8E700BF8034002034
:100F500065630020B034002040420F0070B50D469C
:100F600014461E4602F05EFD50B9022E10D1012C2F
:100F70000ED112A3D3E900230120C5E9002307E025
:100F8000282C10D005D8012C09D0052C0FD000201A
:100F900070BD302CFBD10BA3D3E90023ECE70BA3EE
:100FA000D3E90023E8E70BA3D3E90023E4E70BA38D
:100FB000D3E90023E0E700BFAFF30080401DA1208C
:100FC00026812A0B78F6339F93CACD8D9E6AC42161
:100FD000818A46EE26417272DF25D7B7F017304A74
:100FE00039059E5638B505460E4C0021013500F0F6
:100FF00081FCA4F82C55B4F82C0500F063FC78B102
:10100000B4F82C0500F06EFC014648B9B4F82C0584
:1010100000F070FCB4F82C350133A4F82C35EAE765
:1010200038BD00BF305E0020F8B50D4C02260D4FD4
:10103000A4F5805343F8307C237E3BB965692DB11C
:10104000284601F063F8284601F09CF92046A4F5F3
:10105000A65401F05BF8012E00D1F8BD0126E7E7A8
:10106000A05900203C6800082DE9F04F8FB00546DC
:101070000C4600AF02F0D6FC002849D1237E022B9B
:101080001BD1E38A012B18D102F0B2F90646FFF713
:10109000CBFD03464FF4C87006F51676DFF8C08224
:1010A000B3FBF0F202FB103316FA83F3C8F80030FA
:1010B000E37E33B9A34B00221A703C37BD46BDE82E
:1010C000F08F07F12401204600F04AFE0028F4D1F9
:1010D00007F11400FFF7C0FD97F8264007F114014F
:1010E00007F12700224605F013FB0028E2D10F2C60
:1010F00008D8944B1C70D8F80030A3F51673C8F8C4
:101100000030DAE797F82410284602F083FCD4E791
:10111000E38A282B2BD010D8012B23D0052BCCD140
:10112000BFF34F8F8849894BCA6802F4E0621343CA
:10113000CB60BFF34F8F00BFFDE7302BBDD1844E96
:10114000E17E327A9142B8D1607E3146002291F838
:10115000DC50854200F0A580013201F58A71042A35
:10116000F5D1AAE721462846FFF786FDA5E72146E7
:101170002846FFF7EDFDA0E7B2F8EC507B6005F1E3
:1011800003094FEA99094FEA8902D11DC908A8EB62
:10119000C10300219D46EB46584600F025FC04F1B2
:1011A000EE012A465846314400F00CFC7B6813B926
:1011B000012000F077FB96F8D20000F083FB044694
:1011C00030B9307200F0A8FB204600F06BFBB1E0B4
:1011D000D6F8D4203AB996F8D200B6F82C25824237
:1011E00001D8FFF7FFFED6F8D4202A44944208D253
:1011F00096F8D200B6F82C250130824201D8FFF7CC
:10120000F1FE5FFA89F25946706800F0F5FB08B903
:10121000C54679E0726896F8D2002A447260D6F822
:10122000D42005EB0209C6F8D49000F04BFB8145B1
:1012300009D396F8D220D6F8D4000132001B86F8E4
:10124000D220C6F8D400FF2D0FD80024347200F04D
:1012500063FB204600F026FB00F0DAFE3D4B1881D0
:1012600008B9FFF7ABF9C54627E7BB6896F8D90080
:101270000AFB0362FB68D2F8E41082F8E83001F55B
:101280008061C2F8E030C2F8E410FFF7BFFDFFF75D
:101290000DFE96F8D920013202F0030286F8D9201B
:1012A000B6E74FF48A7A20460AFB02F505F1EA0117
:1012B000314400F051FEF86000287FF4FEAE0122B8
:1012C000354485F8E82002F093F8D5F8E020D6ED13
:1012D000007A801A40F6B832B8EE677ADFED1E6AFF
:1012E000192838BF1920904228BF104607EE900AEF
:1012F000F8EEE77A67EEA67ADFED186AE7EE267A6F
:10130000FCEEE77AC6ED007A96F8D930BB60BA6891
:1013100073680AFB02F4321992F8E81059B1D2F856
:10132000E410E8468B423FF427AF002182F8E81032
:10133000C2F8E010C5467368064A9B0A0133138160
:10134000BBE600BF7934002000ED00E00400FA05A0
:10135000305E002068240020CDCCCC3D6666663F20
:101360007C340020014B1870704700BF74240020AB
:1013700038B54FF00054144B22689A4222D1607D58
:10138000F8B1124B0025C922114918701148237D6C
:101390000930C0F8DB5000F8013C4FF48073C0F80E
:1013A000EF314FF40073C0F803334FF44073C0F8CB
:1013B000173400F007FBE0222946204600F014FB1A
:1013C000012038BD0020FCE79AAD44C574240020FC
:1013D00016000020305E002037B500F019FE1F4CCB
:1013E0001F4D022301221F496B712368288120466B
:1013F0005B68984704F5805301221A49D3F8C0343A
:1014000004F5A6505B689847002317494FF48052B3
:101410000193164B16480093164B02F0D3FA164B65
:10142000197811B1124802F0F5FA01F0E1FF044613
:10143000FFF7FAFB4FF4C873B0FBF3F202FB1303A0
:1014400004F5167010FA83F00C4B186004F09EFB44
:1014500008B10F232B8103B030BD00BFB034002092
:101460006824002040420F00782400205D0F00080F
:101470008034002069100008742400207C3400208F
:101480002DE9F04F00242DED028B93B00DF12C08C7
:101490004FF0010ADFF814B2FFF708FD0A94ADF827
:1014A00034400B94C8F804409FED798B00267E4DA4
:1014B00037462B680DF11D0207A928468DF81CA0A0
:1014C0008DF81D408DED008BD3F808900023C847A0
:1014D0009DF81C90B9F1000F1ED0102200210EA81B
:1014E00000F082FA2B6808AA0AA95F6928460DF164
:1014F0001E03B8470FAB4F4698E8030083E803008C
:101500009DF834300EA958468DF844300A9B0E934E
:10151000DDE9082302F038FD06F5A66605F5A655B7
:10152000B6F5266FC5D1002FC0D1604802F07AFA17
:1015300000283FD15E4E01F05BFF3368984239D3FB
:1015400001F056FF0546FFF76FFB4FF4C8738DF8A7
:101550002870B0FBF3F202FB130305F5167010FAC6
:1015600083F03060534E377817B901238DF8283057
:10157000C7F110050EA8FFF76FFB0EABEDB20DF132
:101580002900D919062D28BF06252A46013500F065
:1015900019FA0AABEDB24548039318230495029358
:1015A000454B0193012300933BA3D3E9002302F0B1
:1015B0007FFA347001F01CFF404A414D1368C31A92
:1015C000B3F57A7F2FD3106001F014FF02460B466B
:1015D000364802F005FB354802F024FA18B32B7A9E
:1015E0000EAF384E002B14BF03230223737101F09A
:1015F000FFFE4FF47A7301223946B0FBF3F03060FE
:10160000304600F085FB182380B202932E4B0193E5
:1016100040F25513CDE903700093244820A3D3E989
:10162000002302F045FA2B7A93B101F0E1FE002687
:1016300007464FF48A7895F8D900304400F003004B
:1016400008FB005393F8E82072B10136042EF2D162
:10165000C82003F005FE2B7A002B7FF417AF13B0E0
:10166000BDEC028BBDE8F08FD3F8E02042B12B68CF
:10167000BA1AFA2B38BFFA230533B2EB430FE4D37F
:10168000FFF7C4FB0028E0D1E2E700BFAFF3008022
:101690000000000000000000401DA12026812A0B50
:1016A000F1C6A7C1D068080FB034002080340020F4
:1016B0007C340020793400207834002060630020DE
:1016C000305E0020682400206463002010B5074CC1
:1016D000204601F051F904F5A65001F04DF9044AF5
:1016E00004490020BDE8104004F0FEBFB0340020E3
:1016F000C063002029100008F8B50A25204C0122FB
:101700004FF400712046192703F0F0F8204601221B
:101710004FF4807103F0EAF84FF4807665200138C9
:1017200025D00822A2F10801B646332905D84FF08A
:10173000000C66834FF000730DE0A1F13403668363
:10174000B3FBF7FC07FB1C33002B0CBF4FF0010C65
:101750004FF0000CEED1013143EA4C238A42A361E1
:10176000A4F818E0E1D10832A02AD8D0DAE7013D88
:1017700042F2107003F074FD15F0FF05BFD1F8BD03
:10178000000402582DE9F84F4FF47A7306460D46CF
:10179000002402FB03F7DFF85080DFF8509098F93F
:1017A00000305FFA84FA5A1C01D0A34212D159F8D2
:1017B00024002A4631460368D3F820B03B46D84778
:1017C000854207D1074B012083F800A0BDE8F88FC0
:1017D0000124E4E7002CFBD04FF4FA7003F040FD45
:1017E0000020F3E7AC630020182300201C23002016
:1017F000002307B5024601210DF107008DF80730DF
:10180000FFF7C0FF20B19DF8070003B05DF804FBAF
:101810004FF0FF30F9E700000A46042108B5FFF752
:10182000B1FF80F00100C0B2404208BD074B0A463C
:1018300030B41978064B53F82140014623682046FE
:10184000DD69044BAC4630BC604700BFAC63002090
:101850001C230020A086010070B5104C0025104EFE
:1018600003F0CEFE20803068238883420CD8002508
:101870002088013803F0C0FE23880544013BB5F5FC
:10188000802F2380F4D370BD03F0B6FE3368054487
:101890000133B5F5802F3360E5D3E8E7AE63002070
:1018A0006863002003F07ABF00F1006000F580203B
:1018B0000068704700F10060920000F5802003F09E
:1018C000FBBE0000054B1A68054B1B889B1A834220
:1018D00002D9104403F090BE0020704768630020D6
:1018E000AE630020024B1B68184403F08BBE00BFA0
:1018F00068630020024B1B68184403F095BE00BFCC
:10190000686300200020704700F1FF5000F58F1041
:10191000D0F8000870470000064991F8243033B130
:1019200000230822086A81F82430FFF7C3BF012092
:10193000704700BF6C630020014B1868704700BF00
:101940000010005C194B01380322084470B51D6873
:10195000174BC5F30B042D0C1E88A6420BD15C68F7
:101960000A46013C824213460FD214F9016F4EB170
:1019700002F8016BF6E7013A03F10803ECD181426A
:101980000B4602D22C2203F8012B0424094A1688A4
:10199000AE4204D1984284BF967803F8016B013CB3
:1019A00002F10402F3D1581A70BD00BF0010005CB0
:1019B00024230020C867000870470000704700001B
:1019C00070470000002310B5934203D0CC5CC45490
:1019D0000133F9E710BD000003460246D01A12F9A0
:1019E000011B0029FAD1704702440346934202D0FA
:1019F00003F8011BFAE770472DE9F8431F4D144621
:101A00000746884695F8242052BBDFF870909CB3B7
:101A100095F824302BB92022FF2148462F62FFF78A
:101A2000E3FF95F824004146C0F1080205EB800071
:101A3000A24228BF2246D6B29200FFF7C3FF95F814
:101A40002430A41B17441E449044E4B2F6B2082E7E
:101A500085F82460DBD1FFF75FFF0028D7D108E0CD
:101A60002B6A03EB82038342CFD0FFF755FF002898
:101A7000CBD10020BDE8F8830120FBE76C63002098
:101A8000024B1A78024B1A70704700BFAC630020FB
:101A90001823002010B5074C4FF4E13306492068A5
:101AA0000B6003F0A5FA60680349BDE8104003F03D
:101AB0009FBA00BF1C23002094630020094B18220A
:101AC000002110B504461846FFF78EFF064A074B63
:101AD00001461278046053F82200BDE8104003F07C
:101AE00087BA00BF94630020AC6300201C23002051
:101AF000F8B571B6002301201A46194602F0A8FE77
:101B00000446802003F0E8FE002849D00025254A3D
:101B100080274FF4D06C3D26136913F0C06F26D197
:101B2000D2F8103113F0C06F21D1236805F10061A4
:101B300099602368D86023685F602368C3F800C099
:101B400021680B6843F001030B6021680B6823F0E8
:101B50001E030B6021680B68DB07FCD4237B8035F8
:101B6000616806FA03F3B5F5001F0B60D4D1204677
:101B700002F0A4FEB5F5001F11D000240A4E0B4D53
:101B8000012003F00BFE3388A34205D928682044C6
:101B9000013403F049FDF6E7002003F0FFFD61B6D4
:101BA000F8BD00BF00200052AE6300206863002033
:101BB0002DE9F3470D46044600219046284640F2A1
:101BC0007912FFF711FF234620220021284604F155
:101BD000220702F07BF9231D022220212846C0267D
:101BE00002F074F9631D03222221284602F06EF9E7
:101BF000A31D03222521284602F068F904F10803F9
:101C000010222821284602F061F904F1100308226D
:101C10003821284602F05AF904F111030822402124
:101C2000284602F053F904F11203082248212846FD
:101C300002F04CF904F1140320225021284602F04E
:101C400045F904F1180340227021284602F03EF9BC
:101C500004F120030822B021284602F037F904F1EC
:101C600021030822B821284602F030F9314608360F
:101C70003B4608222846013702F028F9B6F5A07F36
:101C8000F4D194F83230314604F1330A00268DF84D
:101C9000073008220DF10703284602F017F99DF8D6
:101CA00007304FEAC6099E4209F5A47720D394F87D
:101CB0003231502B28BF50238DF80730B8F1000F78
:101CC00008D1394609F24F170DF1070307222846BC
:101CD00002F0FCF8002604F233149DF8073007EBFD
:101CE000C6019E420DD30731C80802B0BDE8F08797
:101CF0000AEB0603082239462846013602F0E6F8C8
:101D0000CDE7A31908222846013602F0DFF8E4E700
:101D100013B50446084600212022234601900160A5
:101D2000C0F8031002F0D2F8231D019802222021EE
:101D300002F0CCF8631D01980322222102F0C6F8BC
:101D4000A31D01980322252102F0C0F8019804F197
:101D500008031022282102F0B9F8072002B010BDB4
:101D6000F7B5047F05460E462CB1838A122B02D9A3
:101D7000012003B0F0BD0023072228460096194633
:101D800001F068FF731C01220721009328460023FD
:101D900001F060FFD4B9B31C052208212846009346
:101DA00023460D2401F056FFB378102BE0D83746B8
:101DB000BB1BB278934210D307342B7FA88AE40868
:101DC000B3B9844294BF00200120D2E7AB8A082433
:101DD000DB00083BDB08B370E6E7FB1C214608226A
:101DE0002846009300230834013701F033FFDFE772
:101DF000201A18BF0120BCE7F7B5047F05460E4640
:101E00002CB1838ACA2B02D9012003B0F0BD002374
:101E1000082228460096194601F01CFF731CD4B90D
:101E200008220093234610241146284601F012FF91
:101E30007378C82BE8D801235F1C7278013B93426A
:101E400010D307342B7FA88AE408B3B9844294BF27
:101E500000200120D9E7AB8A0824DB00083BDB081F
:101E60007370E5E7F3192146082228460093002302
:101E700001F0F0FE08343B46DEE7201A18BF0120CF
:101E8000C3E70000F7B50D46044600211646284674
:101E90008122FFF7A9FD234608220021284602F0EF
:101EA00015F894F901206378002AB8BF7F238DF8D4
:101EB00007309EB90F270DF1070307220821284696
:101EC00002F004F8002602349DF8073007EBC60143
:101ED0009E4205D30731C80803B0F0BD0827F1E7DB
:101EE000A31908222846013601F0F0FFECE70000B4
:101EF000F7B50E460546002114463046CE22FFF7C0
:101F000073FD2B4628220021304601F0DFFF2B7A9B
:101F1000C82B28BFC8238DF807308CB930240DF1A9
:101F2000070308222821304601F0D0FF2F467B1BF3
:101F30009DF80720934205D3E01DC00803B0F0BD13
:101F40002824F3E707F10903214608223046083424
:101F5000013701F0BBFFEAE7F7B5047F05460E46FF
:101F600034B1838AB3F5827F02D9012003B0F0BD7A
:101F70000123102200212846009601F06BFEDCB9F7
:101F8000B31C09221021284600932346192401F08E
:101F900061FE7388B3F5807FE7D83746BB1B728834
:101FA000934210D307342B7FA88AE408B3B9844244
:101FB00094BF00200120D9E7AB8A1024DB00103B3E
:101FC000DB087380E5E73B1D214608222846009385
:101FD00000230834013701F03DFEDFE7201A18BF67
:101FE0000120C3E730B50A44084D91420DD011F8E5
:101FF000013B5840082340F30004013B2C4013F000
:10200000FF0384EA5000F6D1EFE730BD2083B8ED3E
:10201000F7B5384A6B46106851686A4603C308230F
:102020003549364804F084FB0446002833D10A259C
:10203000334A6B46106851686A4603C30823314926
:102040002E4804F075FB0446002849D00369B3F517
:10205000E01F45D8B0F8661040F2134291423FD1DC
:10206000294A024402F15C018B4239D35C3B23498B
:1020700000209E1AFFF7B6FF04F1640107463246BE
:102080000020FFF7AFFFA3689F4229D1E368984281
:1020900008BF002524E00369B3F5E01F27D8418B72
:1020A00040F21342914220D1174A024402F110013A
:1020B0008B4218D3103B114900209D1AFFF792FF65
:1020C00004F1180106462A460020FFF78BFFA3689B
:1020D0009E4202D1E368984201D00D25A8E7002571
:1020E000284603B0F0BD1025A2E70C25A0E70B257C
:1020F0009EE700BFD8670008DCFF1B000000040853
:10210000E167000890FF1B000800FCF710B5037C96
:10211000044613B9006803F013FC204610BD00000C
:102120000023BFF35B8FC360BFF35B8FBFF35B8F95
:102130008360BFF35B8F7047BFF35B8F0068BFF3B3
:102140005B8F704770B505460C30FFF7F5FF04460E
:1021500005F108063046FFF7EFFFA04206D96D688B
:102160003046FFF7E9FF2544281A70BD3046FFF7D7
:10217000E3FF201AF9E7000070B505464068A0B1FA
:1021800005F10C0605F10800FFF7D6FF04463046BE
:10219000FFF7D2FF844204F1FF34304694BF6D68EC
:1021A0000025FFF7C9FF2C44201A70BD38B50C4636
:1021B0000546FFF7C7FFA04210D305F10800FFF75F
:1021C000BBFF04446868BFF35B8FB4FBF0F100FB16
:1021D00011440120AC60BFF35B8F38BD0020FCE7E9
:1021E0002DE9F041144607460D46FFF7C5FF84422E
:1021F00028BF0446D4B1B84658F80C6B4046FFF7E8
:102200009BFF3044286040467E68FFF795FF331AF5
:102210009C4203D801206C60BDE8F081A41B6B6078
:102220003B682044AB60E8600220F5E72046F3E716
:1022300038B50C460546FFF79FFFA04210D305F1C5
:102240000C00FFF779FF04446868BFF35B8FB4FBB1
:10225000F0F100FB11440120EC60BFF35B8F38BD4F
:102260000020FCE72DE9FF418846694607466C4699
:10227000FFF7B6FF002506B204EBC606B4420AD04B
:10228000626808EB050120680834FFF79BFB54F8EF
:10229000043C1D44F2E729463846FFF7C9FF2846AB
:1022A00004B0BDE8F0810000F8B505460C300F46DB
:1022B000FFF742FF05F1080604463046FFF73CFFF2
:1022C000A042304688BF6C68FFF736FF201A38609E
:1022D00020B12C683046FFF72FFF2044F8BD0000E6
:1022E00073B5144606460D46FFF72CFF8442019055
:1022F00028BF0446DCB101A93046FFF7D5FF019B9A
:1023000033B93268C5E90233C5E9002401200CE085
:102310009C42286038BF0194019884426860F5D9D6
:102320003368241A0220AB60EC6002B070BD204616
:10233000FBE700002DE9FF410F4669466C46FFF7B9
:10234000CFFF00B2002604EBC005AC4209D0D4F8A0
:102350000480B81954F8081B42464644FFF732FB84
:10236000F3E7304604B0BDE8F081000038B505461B
:10237000FFF7E0FF044601462846FFF717FF204617
:1023800038BD000008B103F0DBBA704770470000A9
:1023900010B41346026814680022A4465DF8044B8A
:1023A0006047000000F5805090F859047047000025
:1023B00000F5805090F852047047000000F58050FE
:1023C00090F95804704700004E207047302383F383
:1023D000118800F58052D2F89C34D2F89804184441
:1023E000D2F894341844D2F87C341844D2F88C349F
:1023F0001844D2F888341844002383F311887047B6
:1024000000F58050C0F85414012070472DE9F04FBA
:102410000C4600F5805185B01F4691F852340546B0
:102420009046BDF838909BB1D1F878340133C1F8AB
:1024300078342368980006D4237B082B0BD9627B61
:102440000AB10F2B07D9D1F87C340133C1F87C34A1
:102450004FF0FF3010E0302383F31188EB6AD3F89C
:10246000C42012F4001B0AD0D1F8803400200133BC
:10247000C1F8803480F3118805B0BDE8F08F206882
:102480004822D3F8C4300028C3F3044A6B6AB4BFAF
:1024900040F08040800412FB0A334FEA4A1618606D
:1024A000226852004FEA0A6244BF40F000501860B0
:1024B000207B42EA00425A60607B10B342F4401233
:1024C0005A60D1F8B0240132C1F8B024AA1902F53B
:1024D0008352117B41F020011173207B039300F0A4
:1024E000E3FF0330039B80105FFA8BF20BF1010BCB
:1024F00082420DDA04EB820103EB820249689160AB
:10250000F2E7AA1902F58352117B60F34511E3E764
:102510000122EB6A05EB4A1102FA0AF201F5825137
:10252000C3F8D020AB19183104F10C0203F5825323
:10253000C3E90487234653F8040B934241F8040B84
:10254000F9D11B882E440B8041F2680346F803A0A2
:1025500006F5805609F0030396F86C2043F010034B
:1025600022F01F02134386F86C30002383F3118896
:1025700042463B4621462846CDF8009000F05AFFDF
:10258000012079E72DE9F04700F58056044696F8DA
:102590005254002D40F00381037C032B40F09480C3
:1025A00028462B462F465FFA80FC944510DA01EB53
:1025B000CC0E51F83CC0BCF1000F04DBDEF804C0C7
:1025C000BCF1000F02DB01370130ECE70133FBE720
:1025D000302080F31188E06AF3B9D0F8803043F0FE
:1025E0000203C0F880304E23E06A002F6FD1D0F88C
:1025F000803043F00103C0F880306A4B6A4A1B68A0
:1026000003F1805303F52C539B009342A36240F2E5
:10261000B080664800F0E6FE4D2B42D8DFF884819A
:102620004FEA034EDFF88891D8F800C04EEA8C0ECE
:10263000C0F884E00CF1805000F52C5080006061FF
:1026400003EB0C00D4F82CC0C3F14E03C8F8000013
:10265000DCF8800040F03000CCF880004FF0000C37
:10266000D4F81480E6465FFA8CF08242BCDD01EBC0
:10267000C00A51F83000002810DBDAF804A0BAF1E3
:10268000000F0BDA09EA00400AF07F0A40EA0A006C
:1026900040F0084048F82E000EF1010E0CF1010C3C
:1026A000E1E7836923F00103836100F0A1FE0646A0
:1026B000E36A9B69D90704D500F09AFE831BFA2BC5
:1026C000F6D9002383F311882846BDE8F087B7EBDD
:1026D000530F3DD2DFF8CCE04FEA074CDEF8003074
:1026E0004CEA830CC0F888C003F1805003EB470329
:1026F000002700F52C50CEF80030BC468000A061C9
:10270000E06AD0F8803043F00C03C0F88030D4F891
:1027100018E0FBB29A427FF770AF51F8330001EB3B
:10272000C3080028D8F8043001DB002B0EDB20F0B2
:10273000604023F0604340F0005043F000434EF807
:102740003C000EEBCC000CF1010C43600137E0E7DC
:10275000836923F00103836100F04AFE0646E36AC1
:102760009B69DA07ADD500F043FE831BFA2BF6D93F
:10277000A7E7E26A936923F00103936100F038FE52
:102780000746E36A9B69DB0705D500F031FEC31BF2
:10279000FA2BF6D995E7012586F8525491E70025E2
:1027A00092E700BFBC630020FCB50040EC67000866
:1027B0000000FF0713B500F580540191606CFFF72E
:1027C000DBFC1F280AD920220199606CFFF74AFD23
:1027D000A0F120035842584102B010BD0020FBE791
:1027E00008B5302383F3118800F58050406CFFF763
:1027F00097FC002383F3118808BD000000220260CB
:1028000082814260826070470022002310B5C0E9D7
:102810000023002304460C3020F8043CFFF7EEFFB1
:10282000204610BD2DE9F0479A4688B007468846F5
:102830009146302383F3118807F580546846FFF7EB
:10284000E3FF606CFFF77EFC1F282ED9202269462B
:10285000606CFFF78BFD202827D194F8523423B306
:1028600003AD444605AB2E46083403CE9E4244F8E1
:10287000080C44F8041C3546F5D130682060B38854
:10288000A380DDE90023C9E90023BDF80830AAF8D8
:102890000030002383F3118853464A4641463846A8
:1028A00008B0BDE8F04700F0B3BD002080F3118808
:1028B00008B0BDE8F08700002DE9F84F0023064678
:1028C00000F58154054688461034C0E90133274B92
:1028D00046F8303B374638462037FFF795FFA7428A
:1028E000F9D105F580544FF4805305F5A3594FF005
:1028F000000A26630026676405F5835709F110096D
:102900004FF0000B1037E663C4E90D36012384F85D
:10291000403084F84830A7F11800203747E910AB61
:10292000FFF76CFF47F8286C4F45F4D1B8F1010F61
:1029300084F85884A4F85A64A4F85C64A4F85E642B
:1029400084F86064A4F86264A4F86464A4F866641B
:1029500084F8686402D9064800F044FD054B284617
:1029600053F82830EB62BDE8F88F00BF3C680008E0
:10297000106800082C680008044B10B5197804464C
:102980004A1C1A70FFF798FF204610BDB96300205B
:102990002DE9F04300295AD02E4E2F48B6FBF1F412
:1029A00081428CBF0A201120431EB4FBF0F700FBCC
:1029B0001740DDB220B1022B1846F5D8002032E0D6
:1029C0007B1EB3F5806F2ED2C5EBC5084FF47A732A
:1029D00008F103044FEAE40EC4F3C7040EF1010941
:1029E000281B0EFB033E5FFA80FC59FA80F0BEFB09
:1029F000F0F0B0F5617F18DC83B2601C5CFA80F007
:102A00007843B6FBF0F08142D8D1611E0F29D5D8AA
:102A10000CF1FF310729D1D80120138057801071A4
:102A2000547182F806C0BDE8F08308F1FF34E0106D
:102A3000C4F3C70400F1010E2D1B00FB03335FFA42
:102A400085FC5EFA85F5B3FBF5F39BB2D5E7084646
:102A5000E9E700BF00B4C4043F420F0030B50D4B9E
:102A600005200D4D1C786C438C420ED15978012005
:102A7000518099785171D9789171197911715B7977
:102A800003EB83035B00138030BD013803F10603C1
:102A9000E8D1F9E77C68000840420F0038B540F201
:102AA0007772C36A154CC3F8BC200722C36AC3F807
:102AB000C8202268C16A930043F4C023C1F8A03043
:102AC00002F1805302F16C01C56A03F52C53EA321E
:102AD00089009B00226041F0E061094AC361C5F8AA
:102AE000C01003F5D87103F56A73416293428362A3
:102AF00002D9044800F076FC38BD00BFBC6300205A
:102B0000FCB50040EC6700082DE9F04F00F580555A
:102B10001F4689B0044695F8583489469046022BE2
:102B200004D90026304609B0BDE8F08FA84A52F813
:102B3000231009B942F82300A648C4F80C90017884
:102B40002774C9B9302383F31188A34BD3F8EC2041
:102B500042F48072C3F8EC20D3F8942042F48072DF
:102B6000C3F89420D3F8942022F48072C3F8942000
:102B70000123037081F3118895F851347BB9302318
:102B800083F31188954A95F85834D35C0BB3012B25
:102B900028D0012385F85134002383F31188302392
:102BA00083F31188E26A936923F01003936100F0C4
:102BB0001FFC8246E36A9E6916F0080619D000F0F1
:102BC00017FCA0EB0A03FA2BF4D9002686F3118830
:102BD000A8E70321132002F03FF80321152002F09B
:102BE0003BF8D6E70321142002F036F80321162023
:102BF000F5E79A6942F001029A6100F0F9FB82461A
:102C0000E36A9A69D00706D400F0F2FBA0EB0A034E
:102C1000FA2BF5D9D9E79A694FF0000A42F002027F
:102C20009A61E36AC3F854A08AF3118804F5825BC1
:102C3000686CFFF775FA0BF1100B20220021684633
:102C4000FEF7D2FE02A8FFF7D9FD6A460BEB06039A
:102C50000DF1180ECDF818A094460833BCE8030017
:102C6000F44543F8080C43F8041C6246F4D1DCF840
:102C7000000020361860B6F5806F9CF804201A71A9
:102C8000DBD1002304F5A252494620461A3285F8CA
:102C9000503485F85334FFF77BFE064690B9E26A5C
:102CA000936923F00103936100F0A2FB0546E36AF8
:102CB0009B69D9077FF535AF00F09AFB431BFA2BD0
:102CC000F5D92EE795F85E34C5F86C94591E95F841
:102CD0005F34E26A013B1B0243EA416395F86014EA
:102CE00001390B43B5F85C14013943EA0143D36160
:102CF000B8F1000F36D004F5A35241462046023207
:102D0000FFF7ACFE90B9E26A936923F00103936187
:102D100000F06EFB0546E36A9B69DA077FF501AFB9
:102D200000F066FB431BFA2BF5D9FAE695F8672409
:102D3000C5F87084511E95F86824E36A013A1201BF
:102D400042EA012295F8661401390A43B5F8641481
:102D5000013942EA014242F40002DA604FF4206293
:102D6000E36A9A64E36A4FF000082046C3F8BC8027
:102D7000FFF794FE85F859846FF04042E36A1A65C4
:102D8000174AE36A5A654FF00222E36A9A654FF0E8
:102D9000FF32E36AC3F8E0200322E36A9742DA6570
:102DA0003FF4C0AEE26A936923F00103936100F03F
:102DB0001FFB0746E36A9B69DB0705D500F018FB9C
:102DC000C31BFA2BF6D9ACE6012385F85234A9E6E9
:102DD000B0630020B8630020004402582468000853
:102DE000550200022DE9F04F054689B090469946FC
:102DF000002741F2680A00F58056EB6AD3F8D83014
:102E0000FB40D80751D505EB47124FEA471B524408
:102E10001379190749D4D6F884340133C6F88434B9
:102E200005F5A553C3E9008913799A0605EB0B0252
:102E300048BFD6F8B434524444BF0133C6F8B43462
:102E4000137943F008031371DB0723D596F8533445
:102E500003B305F582546846FFF7D6FC03AB18347C
:102E60005C4404F1080C2068083454F8041C1A4629
:102E7000644503C21346F6D12068694610602846AF
:102E8000A2889A800123ADF808302B68CDE900892B
:102E9000DB6B9847D6F8A834D6F854040133C6F84B
:102EA000A83410B103681B6998470137202FA4D1BB
:102EB00009B0BDE8F08F00002DE9F04F0F468DB04E
:102EC000044600F097FA82468946002F5BD1E36AF8
:102ED000D3F8A02012F4FE0F03D100200DB0BDE8FE
:102EE000F08FD3F8A420920141BF04F58051D1F8AE
:102EF00098240132C1F89824D3F8A4205606ECD0C7
:102F0000D3F8A450E669C5F305254823E8464FF0F9
:102F1000000B03FB05664046FFF770FC326851006A
:102F20004ABF22F06043C2F38A4343F00043920059
:102F300048BF43F080430093736813F400131BBF32
:102F4000012304F580528DF80D308DF80D301EBF31
:102F5000D2F8B8340133C2F8B834F38803F00F0361
:102F60008DF80C309DF80C0000F09EFA5FFA8BF3A0
:102F7000984225D9F2180CA90BF1010B127A0B44D7
:102F800003F82C2CEEE7012FA7D1E36AD3F8B02089
:102F900012F4FE0FA1D0D3F8B420950141BF04F57F
:102FA0008051D1F898240132C1F89824D3F8B42084
:102FB000500692D0D3F8B450266AC5F30525A4E78D
:102FC000EFB9E36AC3F8A85004A807ADFFF71CFCEB
:102FD00098E80F0007C52B800023204604A9ADF810
:102FE0001830236804F58054DB6BCDE904A99847B9
:102FF00058B1D4F890340133C4F890346EE7012FFF
:10300000E2D1E36AC3F8B850DEE7D4F89434012083
:103010000133C4F8943461E72DE9F04105460F46C9
:1030200000F58054012639462846FFF745FF10B1C8
:1030300084F85364F7E7D4F8A834D4F8540401337F
:10304000C4F8A83420B10368BDE8F0411B691847F3
:10305000BDE8F081C36AF0B51A6C12F47F0F2BD073
:103060001B6C00F5805441F268054FF0010CC4F868
:10307000AC340023471900EB43125E012A44117956
:1030800011F0020F15D0490713D4B959C66A0CFACA
:1030900001F1D6F8CCE011EA0E0F0AD0C6F8D41030
:1030A000117941F004011171D4F88C240132C4F873
:1030B0008C240133202BDED1F0BD00002B4B70B5EA
:1030C0001E561B5C012B30D8294D2A4A55F8233057
:1030D00052F8264013B349B3236D9A0510D54FF427
:1030E0000073236500F086F950EA01020B4602D016
:1030F000013861F10003024655F82600FFF772FE21
:10310000236D9B012CD54FF0007255F826302265B7
:1031100003F58053012283F8592421E0012323651C
:10312000102323654FF48053236570BD236DDA07A8
:1031300002D4236D5B0706D50523002155F8260030
:103140002365FFF769FF236DD80602D4236D590666
:1031500006D55023012155F826002365FFF75CFFB3
:1031600055F82600BDE87040FFF774BF28680008D6
:10317000B06300202C68000808B5302383F3118861
:10318000FFF768FF002383F3118808BDC36AD3F8F3
:10319000C00010F07C5005D0D3F8C40080F40010BB
:1031A000C0F340507047000008B5302383F3118806
:1031B00000F58050406CFEF7C5FF002383F31188B3
:1031C00043090CBF0120002008BD000000F580531A
:1031D00093F8592462B1C16A8A6922F001028A61B6
:1031E000D3F89C240132C3F89C24002283F859248C
:1031F000704700002DE9F743302181F3118800F575
:103200008251002541F2680E4FF00108103100F59F
:10321000805C00EB45147444267977071CD4F606CD
:103220001AD58E69D0F82C9008FA06F6D9F8CC7029
:103230003E4211D04F6801970F689742019F9F410E
:103240000AD2C9F8D460267946F004062671DCF863
:1032500088440134CCF8884401352031202DD8D160
:10326000002383F3118803B0BDE8F083F8B51E4650
:1032700000230F46054613701446FFF795FF80F0B4
:10328000010038701EB12846FFF780FF2070F8BD9E
:103290002DE9F04F85B099460D468046164691F8C7
:1032A00000B0DDE90EA302931378019300F0A2F8B9
:1032B0002B7804460F4613B93378002B41D02246B1
:1032C0003B464046FFF796FFFFF756FFFFF77EFFAE
:1032D0004B4632462946FFF7C9FF2B7833B1BBF185
:1032E000000F03D0012005B0BDE8F08F337813B193
:1032F000019B002BF6D108F5805303935445029BA4
:1033000077EB03031DD2039BD3F85404C8B10368C1
:10331000AAEB04011B6898474B46324629464046B3
:10332000FFF7A4FF2B7813B1BBF1000FDAD133788C
:1033300013B1019B002BD5D100F05CF804460F4679
:10334000DCE70020CFE70000002108B50846FFF7C2
:10335000B5FEBDE8084001F071B8000008B50121D4
:103360000020FFF7ABFEBDE8084001F067B80000A1
:1033700008B500210120FFF7A1FEBDE8084001F0DB
:103380005DB80000012108B50846FFF797FEBDE8CB
:10339000084001F053B8000000B59BB0EFF309817D
:1033A00068226846FEF70EFBEFF30583014B9B6B2B
:1033B000FEE700BF00ED00E008B5FFF7EDFF0000FD
:1033C00000B59BB0EFF3098168226846FEF7FAFA70
:1033D000EFF30583014B5B6BFEE700BF00ED00E000
:1033E000FEE700000FB408B5029801F0E9FEFEE721
:1033F00002F0D4BA02F0B6BA13B56C46031D84E8E5
:10340000060094E8030083E80500012002B010BD27
:1034100073B58568019155B11B885B0707D4D0E966
:1034200000369B6B9847019AC1B23046A8470120ED
:1034300002B070BDF0B5866889B005460C465EB135
:10344000BDF838305B070AD4D0E900379B6B98474A
:103450002246C1B23846B047012009B0F0BD002273
:10346000002301F10806CDE9002300230A46ADF848
:10347000083003AB1068083252F8041C1C46B242F4
:1034800003C42346F6D1106820609288A280FFF71B
:10349000B1FF0423ADF808302B68CDE90001DB6BE8
:1034A000694628469847D7E7082817D909280CD035
:1034B0000A280CD00B280CD00C280CD00D280CD0CE
:1034C0000E2814BF4020302070470C207047102079
:1034D0007047142070471820704720207047000064
:1034E0002DE9F041456A15B94162BDE8F0814B68AC
:1034F000AC4623F06047C3F38A464FEAD37EC3F35A
:10350000807816EA230638BF3E462B465A68BEEB43
:10351000D27F22F060440AD0002A18DAA40CB44208
:1035200017D19D420FD10D60DEE71346EEE7A742AB
:1035300007D102F08044C2F3807242450BD054B1EF
:10354000EFE708D2EDE7CCF800100B60CDE7B4420E
:1035500001D0B442E5D81A689C46002AE5D119602A
:10356000C3E700002DE9F047089D01F0070400EBD8
:10357000D1004FF47F494FEAD508224405F00705F2
:10358000944201D1BDE8F08704F0070705F0070A6F
:10359000111B08EBD50E57453E4613F80EC038BF39
:1035A0005646C6F108068E4228BF0E46E108415C29
:1035B00034443544B94029FA06F721FA0AF1FFB23A
:1035C0008CEA010147FA0AF739408CEA010C03F84A
:1035D0000EC0D5E780EA0120082341F2210201B2A2
:1035E000013B4000002980B2B8BF504013F0FF03F8
:1035F000F5D1704738B50C468D18A54200D138BDBD
:1036000014F8011BFFF7E6FFF7E7000042684AB134
:10361000136881894360438901339BB29942438196
:1036200038BF83811046704770B588B004462022A9
:103630000D4668460021FEF7D7F920460495FFF7AE
:10364000E5FF024660B16B46054608AE1C460835EC
:1036500003CCB44245F8080C45F8041C2346F5D1C8
:10366000104608B070BD0000082817D909280CD0F2
:103670000A280CD00B280CD00C280CD00D280CD00C
:103680000E2814BF4020302070470C2070471020B7
:1036900070471420704718207047202070470000A2
:1036A000082817D90C280CD910280CD914280CD9A3
:1036B00018280CD920280CD930288CBF0F200E20B8
:1036C0007047092070470A2070470B2070470C2074
:1036D00070470D20704700002DE9F843078C044621
:1036E000072F1ED900254FF6FF73D0E90298C5F1C8
:1036F0002006A5F1200029FA05F1083508FA06F69A
:1037000028FA00F0314301431846C9B2FFF762FFBF
:10371000402D0346EBD13A46E169BDE8F843FFF797
:1037200069BF4FF6FF70BDE8F883000010B54B6825
:1037300023B9CA8A63F30902CA8210BD04691A68F0
:103740001C600361C38A013BC3824A60EFE700004B
:103750002DE9F84F1D46CB8A0F468146C3F3090178
:10376000924605290B4630D00020AAB207F11A0470
:103770009EB21FFA80F8042E0FD8904503F1010382
:1037800006D30A44FB8A62F309030120FB821AE094
:103790001AF800600130E654EAE79045F1D2A1F151
:1037A000050B1C237C68BBFBF3F203FB12BB1FFA67
:1037B0008BF6002C45D14846FFF728FF044638B960
:1037C00078606FF00200BDE8F88F4FF00008E6E780
:1037D000002606607860ADB24FF0000B454510D969
:1037E0000AEB0803221D13F8011B08F1010891558B
:1037F000B1B21FFA88F81B292BD0454506F1010606
:10380000F1D8FB8AC3F30902154465F30903BCE749
:1038100001321C4692B22368002BF9D16B1F0B4476
:103820001C21B3FBF1F301339BB29A42D3D2BBF11B
:10383000000FD0D14846FFF7E9FE20B9C4F800B028
:10384000BFE70122E7E7C0F800B05E46206004460B
:10385000C1E74545D5D94846FFF7D8FE08B92060ED
:10386000AFE7C0F800B0002620600446B6E70000CD
:103870002DE9F04F1C46074688462DED028B83B09C
:103880005B690192002B00F09A80238C2BB1E269D6
:10389000002A00F09480072B35D807F10C00FFF7C1
:1038A000B5FE054638B96FF00205284603B0BDECF9
:1038B000028BBDE8F08F14220021FEF795F8228CD0
:1038C000E16905F10800FEF77DF8208C48F0004121
:1038D000013080B2FFF7E4FEFFF7C6FE013880B288
:1038E00020840130287438466369228C1B782A446E
:1038F00003F01F0363F03F03137269602946FFF76B
:10390000EFFD0125D1E74FF0000900F10C034FF066
:10391000800A4E464D4608EE103A18EE100AFFF7A0
:1039200075FE83460028BED014220021FEF75CF805
:10393000002E3AD1019B0222ABF808300BF1080EA1
:103940001FFA82FC218C0CF10100BCF1060F80B241
:1039500001D88E422BD3FFF7A3FE8E4208BF4FF053
:10396000400AFFF781FE62690138013512781BFABF
:1039700080F1013002F01F022DB242EA491289F0B3
:1039800001094AEA020A48F0004281F808A05946B3
:103990008BF810003846CBF804204FF0000AFFF7F0
:1039A0009FFD238CB342B8D17FE70022C6E7E169CF
:1039B000895D01360EF80210B6B20132C0E76FF031
:1039C000010572E7F8B515460E463022002104467F
:1039D0001F46FEF709F8069BB5F5001FA760636058
:1039E00004F11000079B34BF6A094FF6FF72E661CD
:1039F000A362002397B29A4206D800230360A782ED
:103A0000E3822383E360F8BD06600133304620364D
:103A1000F1E7000003781BB94BB2002BC8BF01705F
:103A20007047000000787047F8B50C46C969074632
:103A300011B9238C002B37D1257E1F2D34D838782F
:103A400028BB228C072A2CD8268A36F003032BD1D8
:103A50004FF6FF70FFF7CEFD20F0010031024FF668
:103A6000FF72400441EA0561400C41EA40252346CB
:103A700029463846FFF7FCFE002807DD6269137807
:103A80000133DBB21F2B88BF00231370F8BD218ADE
:103A90002D0645EA012505432046FFF71DFE024697
:103AA000E5E76FF00300F1E76FF00100EEE70000DB
:103AB00070B58AB0044616460021282268461D4685
:103AC000FDF792FFBDF8383069462046ADF810305A
:103AD0000F9B05939DF840308DF81830119B07938C
:103AE000BDF84830CDE90265ADF82030FFF79CFF06
:103AF0000AB070BD2DE9F041D36905460C46164663
:103B00000BB9138C5BBB377E1F2F28D895F800802C
:103B1000B8F1000F26D03046FFF7DEFD33782102E2
:103B20000246284641EAC331338A41EA080141EAA4
:103B3000076141EA0341334641F08001FFF798FEF7
:103B400000280ADD3378012B07D17269137801331D
:103B5000DBB21F2B88BF00231370BDE8F0816FF02C
:103B60000100FAE76FF00300F7E70000F0B58BB053
:103B700004460D4617460021282268461E46FDF7DA
:103B800033FF9DF84C30294620465A1E534253417C
:103B90006A468DF800309DF84030ADF81030119B2A
:103BA00005939DF848308DF81830149B0793BDF8A5
:103BB0005430CDE90276ADF82030FFF79BFF0BB013
:103BC000F0BD0000406A00B104307047436A1A68D3
:103BD000426202691A600361C38A013BC382704773
:103BE0002DE9F041D0F8208014461D46184E41467C
:103BF000002709B9BDE8F081D1E90223A21A65EBDB
:103C00000303964277EB03031ED2036A8B420DD166
:103C1000FFF78CFD036A1B68036203690B60C38AAC
:103C20000161013B016AC3828846E2E7FFF77EFD3E
:103C30000B68C8F8003003690B60C38A0161013B5F
:103C4000C382D8F80010D4E788460968D1E700BFDE
:103C500080841E002DE9F04F8BB00D4614469B4624
:103C6000DDF850908046002800F01881B9F1000F6F
:103C700000F01481531E3F2B00F21081012A03D162
:103C8000BBF1000F40F00A810023CDE90833B8F8FA
:103C90001430B5EBC30F4FEAC30703D300200BB0BA
:103CA000BDE8F08F2B199F42D8F80C3036BF7F1B30
:103CB0002746FFB21BB9D8F81030002B7AD0272D39
:103CC0004DD8C5F1280600232946B742009308AB1A
:103CD000D8F808002CBFF6B23E46A7EB060A3544DA
:103CE00032465FFA8AFAFFF73DFCB8F81430282113
:103CF00003F10053053BDB000493D8F80C30039329
:103D0000039B13B1BAF1000F2CD1D8F8100040B1C9
:103D1000BAF1000F05D008AB5246691A0096FFF7BA
:103D200021FC38B2002FB9D066070AD00AAB624234
:103D300003EBD40102F0070211F8083C134101F82B
:103D4000083C082C3DD9102C40F2B580202C40F2C4
:103D5000B780BBF1000F00F09C80082335E0BA4625
:103D60000026C2E7049BE02B28BFE02306930B4408
:103D7000AB42059315D95A1B0398691A00969245D0
:103D800008AB00F1040034BF5246D2B20792FFF7ED
:103D9000E9FB079A1644AAEB020A1544F6B25FFA49
:103DA0008AFA049B069A05999B1A0493039B1B6845
:103DB0000393A5E700933A4608AB2946D8F80800D4
:103DC000ADE7BBF1000F13D00123B4EBC30F6BD0F1
:103DD000082C12D89DF82030621E23FA02F2D50773
:103DE00006D54FF0FF3202FA04F423438DF8203059
:103DF0009DF8203089F8003051E7102C12D8BDF81A
:103E00002030621E23FA02F2D10706D54FF0FF32AE
:103E100002FA04F42343ADF82030BDF82030A9F8AD
:103E200000303CE7202C0FD80899631E21FA03F3D9
:103E3000DA0705D54FF0FF3202FA04F40C43089478
:103E4000089BC9F800302AE7402C2AD0611EC4F133
:103E50002102A4F12103DDE9086526FA01F105FA42
:103E600002F225FA03F311431943CB0711D50122BE
:103E7000A4F12003C4F1200102FA03F322FA01F1B4
:103E8000A2400B43524263EB430332432B43CDE941
:103E90000823DDE90823C9E9002300E76FF00100EA
:103EA000FDE66FF00800FAE6082CA1D9102CB4D971
:103EB000202CEED8C4E7BBF1000FAED0022384E77C
:103EC000BBF1000FBCD004237FE70000012A30B50E
:103ED000144638BF012485B00025402C28BF40245B
:103EE000012ACDE9025518D81B788DF808306307F0
:103EF0000AD004AB624203EBD40502F0070215F8C6
:103F0000083C934005F8083C0346009122460021F6
:103F100002A8FFF727FB05B030BD082AE4D9102A14
:103F200003D81B88ADF80830E1E7202A95BF1B684D
:103F3000D3E900230293CDE90223D8E710B5CB687B
:103F40001BB98B600B618B8210BD04691A681C6001
:103F50000361C38A013BC382CA60F0E703064CBF1A
:103F6000C0F3C0300220704708B50246FFF7F6FFE5
:103F7000022806D15306C2F30F2001D100F003003E
:103F800008BDC2F30740FBE72DE9F04F93B00446AC
:103F90000D46CDE903230A681046FFF7DFFF02282C
:103FA000824614BFC2F306260026002A80F2F8815A
:103FB00012F0C04940F0F481097B002900F0F08143
:103FC000022803D02378B34240F0ED81C2F30463AA
:103FD00010462944069302F07F030593FFF7C4FFC0
:103FE000059B002283464FEA8348002348EA0A489B
:103FF00048EA4668CE78CDE90823F30948EA000884
:10400000029368D0059B024608A9204600935346B8
:104010006768B847002800F0C981276A4FB9414650
:1040200004F10C00FFF700FB074690B96FF00200A7
:1040300055E03B6998450DD03F68002FF9D14146C6
:1040400004F10C00FFF7F0FA07460028EED0236ACF
:104050003B60276297F817C006F01F08CCF3840C6A
:10406000ACEB0800A8EB0C031FFA80FE0028B8BFD9
:104070000EF120001FFA83FEB8BF00B2002B079399
:10408000B8BF0EF12003D7E90221BCBF1BB20793D2
:1040900052EA010338D0039B4FF0000CDFF81CE319
:1040A0009A1A049B63EB010196457CEB01032BD329
:1040B0006B7B97F81AE0734519D1029B002B78D0DF
:1040C000012821DC7868F8B9DFF8ECC2944570EB80
:1040D000010316D337E0276A27B96FF00C0013B03D
:1040E000BDE8F08F3B699845B4D03F68F4E7B2482B
:1040F00090427CEB010301D30020F0E7029B002BF0
:10410000FAD0079B0F2B17DCFA7DB3003946204607
:1041100002F0030203F07C031343FB75FFF706FB79
:104120006B7BBB76029B3BB9FB7DC3F38402013200
:1041300062F38603FB75D0E76A7BBB7E9A42DBD1D4
:10414000029B002B35D0B309022B32D0039B1422E3
:1041500000210DA8BB60049BFB60FDF745FC039BA1
:104160000AA920460A93049BADF83EB00B932B1D81
:104170008DF840A00C932B7B8DF84180013BDBB286
:10418000ADF83C30069B8DF84230059B8DF84330EE
:1041900094F82C3083F001038DF84430A3689847DD
:1041A000FB7DC3F38403013303F01F039B02FB82F7
:1041B000A2E7FB7DC6F34012B2EBD31F40F0F980BB
:1041C000C3F38403434540F0FB80029AB6092B7B7E
:1041D000002A52D016F0010661D1032B40F2F38081
:1041E000039B394604F10C00BB60049BFB60FB8A17
:1041F00066F30903AE1DFB8232462B7B033BDBB229
:10420000FFF7A6FA00280CDA39462046FFF78EFAA7
:10421000FB7DC3F38403013303F01F039B02FB8286
:1042200004E7AB88DDE908843B834FF6FF73C9F1EF
:104230002000A9F1200228FA09F109F1080904FA7D
:1042400000F024FA02F2014318461143C9B2FFF705
:10425000C1F9B9F1400F0346E9D1B88231462A7B52
:10426000033AD2B2FFF7C6F9FB7DB882DA43C2F354
:10427000C01262F3C713FB753EE786B92E1D013BE2
:10428000394604F10C00DBB23246FFF761FA002830
:10429000BADB2A7B3146B88A013AD2B2E2E7F98A20
:1042A000013BC1F30901DAB204295BD8281D0023C0
:1042B00007F11B069A4208D910F801CB013306F822
:1042C00001C00131DBB20529F4D1039993420A916F
:1042D00038BF043304992CBF002355FA83F30B91A4
:1042E00007F11B010C9179680E930D91291DFB8A32
:1042F000ADF83EB0C3F309038DF840A08DF84180BE
:104300001A44069B8DF84230059BADF83C208DF891
:10431000433094F82C3083F001038DF844300023AF
:10432000B88A7B602A7B013AFFF764F93B8BB8823D
:10433000834203D1A3680AA92046984720460AA9C8
:10434000FFF7FCFDFB7DBA8AC3F38403013303F05E
:104350001F039B02FB823B8B9A420CBF00206FF035
:104360001000BCE67B68002BAFD0052001E01C30BC
:1043700033461E68002EFAD1091A2E1D081D184456
:1043800001EB090C5FFA89F3BCF11B0F9DD89A422F
:104390009BD916F8013B09F1010900F8013BEFE751
:1043A0006FF009009BE66FF00A0098E66FF00B00D3
:1043B00095E66FF00D0092E640420F0080841E00EB
:1043C0006FF00E008BE66FF00F0088E6EFF30983C5
:1043D000054968334A6B22F001024A6383F3098876
:1043E000002383F31188704700EF00E0302080F352
:1043F000118862B60D4B0E4AD96821F4E0610904B8
:10440000090C0A430B49DA60D3F8FC2042F08072B1
:10441000C3F8FC20084AC2F8B01F116841F001013E
:1044200011602022DA7783F82200704700ED00E067
:104430000003FA0555CEACC5001000E0302310B5DE
:1044400083F311880E4B5B6813F4006314D0F1EE14
:10445000103AEFF309844FF08073683CE361094B35
:10446000DB6B236684F3098800F070FE10B1064B05
:10447000A36110BD054BFBE783F31188F9E700BF8B
:1044800000ED00E000EF00E03F04000842040008F7
:1044900008B5074B074A196801F03D019960536858
:1044A0000BB190689847BDE80840FFF7C7BF00BF51
:1044B00000000240C463002008B5084B1968890950
:1044C00001F03D018A019A60054AD3680BB1106979
:1044D0009847BDE80840FFF7B1BF00BF00000240A9
:1044E000C463002008B5084B1968090C01F03D01B0
:1044F0000A049A60054A53690BB190699847BDE870
:104500000840FFF79BBF00BF00000240C4630020CB
:1045100008B5084B1968890D01F03D018A059A60BC
:10452000054AD3690BB1106A9847BDE80840FFF708
:1045300085BF00BF00000240C463002008B5074BE0
:10454000074A596801F03D01D960536A0BB1906A7E
:104550009847BDE80840FFF771BF00BF0000024068
:10456000C463002008B5084B5968890901F03D0172
:104570008A01DA60054AD36A0BB1106B9847BDE82F
:104580000840FFF75BBF00BF00000240C46300208B
:1045900008B5084B5968090C01F03D010A04DA60BE
:1045A000054A536B0BB1906B9847BDE80840FFF785
:1045B00045BF00BF00000240C463002008B5084B9F
:1045C0005968890D01F03D018A05DA60054AD36B0F
:1045D0000BB1106C9847BDE80840FFF72FBF00BF34
:1045E00000000240C463002008B5074B074A196861
:1045F00001F03D019960536C0BB1906C9847BDE898
:104600000840FFF71BBF00BF00040240C463002046
:1046100008B5084B1968890901F03D018A019A60C3
:10462000054AD36C0BB1106D9847BDE80840FFF701
:1046300005BF00BF00040240C463002008B5084B5A
:104640001968090C01F03D010A049A60054A536D8E
:104650000BB1906D9847BDE80840FFF7EFBE00BF73
:1046600000040240C463002008B5084B1968890D96
:1046700001F03D018A059A60054AD36D0BB1106EB9
:104680009847BDE80840FFF7D9BE00BF00040240CC
:10469000C463002008B5074B074A596801F03D0183
:1046A000D960536E0BB1906E9847BDE80840FFF794
:1046B000C5BE00BF00040240C463002008B5084B1B
:1046C0005968890901F03D018A01DA60054AD36E13
:1046D0000BB1106F9847BDE80840FFF7AFBE00BFB1
:1046E00000040240C463002008B5084B5968090C57
:1046F00001F03D010A04DA60054A536F0BB1906F77
:104700009847BDE80840FFF799BE00BF000402408B
:10471000C463002008B5084B5968890D01F03D01BC
:104720008A05DA60054AD36F13B1D2F88000984742
:10473000BDE80840FFF782BE00040240C4630020C9
:1047400000230C4910B51A460B4C0B6054F823009B
:10475000026001EB430004334260402BF6D1074A6C
:104760004FF0FF339360D360C2F80834C2F80C34C2
:1047700010BD00BFC46300209C6800080000024018
:104780000F28F8B510D9102810D0112811D01228F0
:1047900008D10F240720DFF8B4E00126DEF800502E
:1047A000A04208D9002649E00446F4E70F2400207F
:1047B000F1E70724FBE706FA00F73D4240D1214C20
:1047C0004FEA001C3D4304EB00160EEBC000CEF890
:1047D0000050C0E90123FBB24BB11B48836B43F08F
:1047E00001038363036E43F001030366036E17F452
:1047F0007F4F09D01448836B43F002038363036E39
:1048000043F002030366036E54F80C00036823F0C0
:104810001F030360056815F00105FBD104EB0C03D1
:104820003D2493F80CC05F6804FA0CF43C6021242A
:104830000560446112B1987B00F00EFA3046F8BD75
:104840000130ADE79C68000800450258C4630020B1
:1048500010B5302484F31188FFF792FF002383F30F
:10486000118810BD10B50446807B00F00BFA0123BF
:104870001049627B03FA02F20B6823EA0203DAB200
:104880000B604AB90C4A916B21F001019163116EE2
:1048900021F001011166126E13F47F4F09D1064B0E
:1048A0009A6B22F002029A631A6E22F002021A66D2
:1048B0001B6E10BDC46300200045025808B53023AC
:1048C00083F31188FFF7CEFF002383F3118808BD1F
:1048D0000023054A19460133102BC2E9001102F1E9
:1048E0000802F8D1704700BF486400202DE9F74F57
:1048F00002F0030AC2F3C313C2F38009C2F3C10872
:10490000C2F3411E574600224FF00F0B0193CB0715
:1049100033D502F00703019C012556009B00BAF134
:10492000020F05FA02F504FA03FC44680BFA03F3DC
:1049300024EA05046FEA030344EA090444604FF0E3
:104940000304856804FA06F625EA06056FEA0604FC
:1049500045EA08058560C56825EA060545EA0E05AD
:10496000C5601BD1072A13D8056A2B4043EA0C0304
:10497000036203681C403C430460490822D04FEAAC
:10498000490901324FEA88084FEA8E0EBF00BEE7A0
:10499000456A2B4043EA0C034362EAE70568072AAD
:1049A00004EA050444EA0704046005D8046A2340C5
:1049B00043EA0C030362E0E7446A234043EA0C0342
:1049C0004362DAE703B0BDE8F08F00000268436895
:1049D0001143016003B1184770470000024A136891
:1049E00043F0C0031360704700100140024A13688F
:1049F00043F0C00313607047007C004037B51A4C89
:104A00001A4D204600F0E8FA04F114000094002347
:104A10004FF40072164900F0A5F94FF400721549E1
:104A200004F138000094144B00F01EFA134BC4E953
:104A30001735134C204600F0CFFA04F11400002380
:104A40004FF400720F49009400F08CF90E4B4FF4B4
:104A500000720E4904F13800009400F005FA0C4B86
:104A6000C4E9173503B030BDC864002000E1F50586
:104A7000A0650020A0690020DD4900080010014069
:104A800034650020A0670020ED490008A06B0020DD
:104A9000007C0040037C30B5284C002918BF0C4630
:104AA000012B0CD1264B984236D1264B1A6D42F081
:104AB00010021A659A6F42F010029A679B6F226883
:104AC000036EC16D03EB52038466B3FBF2F36268BD
:104AD000150442BF23F0070503F0070343EA45032B
:104AE000CB60A36843F040034B60E36843F00103ED
:104AF0008B6042F4967343F001030B604FF0FF3379
:104B00000B62510505D512F0102213D0B2F1805F6F
:104B100012D080F8643030BD0B4B9842CFD1094B96
:104B20009A6C42F000429A641A6F42F000421A678F
:104B30001B6FC4E77F23ECE73F23EAE79C6900088B
:104B4000C864002000450258346500202DE9F04774
:104B5000C66D05463768F469210734621AD014F02F
:104B6000080118BF4FF48071E20748BF41F02001EF
:104B7000A3074FF0300348BF41F04001600748BF32
:104B800041F0800183F31188281DFFF71FFF0023E8
:104B900083F31188E2050AD5302383F311884FF49B
:104BA0008061281DFFF712FF002383F311884FF067
:104BB00030094FF0000A14F0200838D13B0616D512
:104BC0004FF0300905F1380A200610D589F3118815
:104BD000504600F07DF9002836DA0821281DFFF73D
:104BE000F5FE27F080033360002383F311887906F4
:104BF00014D5620612D5302383F31188D5E9132327
:104C00009A4208D12B6C33B127F040071021281DA0
:104C1000FFF7DCFE3760002383F31188E30618D525
:104C2000AA6E1369ABB15069BDE8F047184789F324
:104C30001188736A284695F86410194000F0E6F967
:104C40008AF31188F469B6E7B06288F31188F469D1
:104C5000BAE7BDE8F0870000090100F160430122D6
:104C600003F56143C9B283F8001300F01F039A40B3
:104C700043099B0003F1604303F56143C3F88021BE
:104C80001A60704700F01F0301229A40430900F1A7
:104C900060409B0000F5614003F1604303F5614310
:104CA000C3F88020C3F88021002380F800337047C8
:104CB000F8B51546826804460B46AA4200D28568BC
:104CC000A1692669761AB5420BD218462A46FCF726
:104CD00079FEA3692B44A3612846A3685B1BA360EC
:104CE000F8BD0CD9AF1B18463246FCF76BFE3A46AE
:104CF000E1683044FCF766FEE3683B44EBE71846A6
:104D00002A46FCF75FFEE368E5E70000836893420C
:104D1000F7B50446154600D28568D4E90460361A12
:104D2000B5420BD22A46FCF74DFE63692B44636102
:104D30002846A3685B1BA36003B0F0BD0DD93246C3
:104D4000AF1B0191FCF73EFE01993A46E068314401
:104D5000FCF738FEE3683B44E9E72A46FCF732FEFD
:104D6000E368E4E710B50A440024C361029B846051
:104D7000C16002610362C0E90000C0E9051110BD15
:104D800008B5D0E90532934201D1826882B98268C0
:104D9000013282605A1C426119700021D0E904324C
:104DA0009A4224BFC368436100F076FA002008BD30
:104DB0004FF0FF30FBE7000070B5302304460E468D
:104DC00083F31188A568A5B1A368A269013BA3601C
:104DD000531CA36115782269934224BFE368A36141
:104DE000E3690BB120469847002383F311882846D6
:104DF00007E03146204600F03FFA0028E2DA85F36A
:104E0000118870BD2DE9F74F04460E4617469846A7
:104E1000D0F81C904FF0300A8AF311884FF0000B45
:104E2000154665B12A4631462046FFF741FF034645
:104E300060B94146204600F01FFA0028F1D0002357
:104E400083F31188781B03B0BDE8F08FB9F1000F30
:104E500003D001902046C847019B8BF31188ED1ABF
:104E60001E448AF31188DCE7C160C361009B826045
:104E70000362C0E905111144C0E9000001617047F7
:104E8000F8B504460D461646302383F31188A7680B
:104E9000A7B1A368013BA36063695A1C62611D70DE
:104EA000D4E904329A4224BFE3686361E3690BB139
:104EB00020469847002080F3118807E031462046BD
:104EC00000F0DAF90028E2DA87F31188F8BD000073
:104ED000D0E9052310B59A4201D182687AB9826877
:104EE0000021013282605A1C82611C7803699A4257
:104EF00024BFC368836100F0CFF9204610BD4FF096
:104F0000FF30FBE72DE9F74F04460E46174698465B
:104F1000D0F81C904FF0300A8AF311884FF0000B44
:104F2000154665B12A4631462046FFF7EFFE034697
:104F300060B94146204600F09FF90028F1D00023D7
:104F400083F31188781B03B0BDE8F08FB9F1000F2F
:104F500003D001902046C847019B8BF31188ED1ABE
:104F60001E448AF31188DCE702684368114301603C
:104F700003B11847704700001430FFF743BF00002B
:104F80004FF0FF331430FFF73DBF00003830FFF71C
:104F9000B9BF00004FF0FF333830FFF7B3BF000058
:104FA0001430FFF709BF00004FF0FF311430FFF756
:104FB00003BF00003830FFF763BF00004FF0FF323F
:104FC0003830FFF75DBF0000012914BF6FF01300F8
:104FD00000207047FFF712BD044B036000234360BD
:104FE000C0E9023301230374704700BFB4690008AD
:104FF00010B53023044683F31188FFF74BFD0223DD
:105000000020237480F3118810BD000038B5C369F7
:1050100004460D461BB904210844FFF7A5FF2946A5
:1050200004F11400FFF7ACFE002806DA201D4FF44F
:105030000061BDE83840FFF797BF38BD00238268A4
:10504000037503691B6899689142FBD25A68036033
:1050500042601060586070470023826803750369DE
:105060001B6899689142FBD85A68036042601060DF
:105070005860704708B50846302383F311880A7DCD
:105080000023052A06D8DFE802F00B050503120EFF
:10509000826913604FF0FF338361FFF7CFFF002376
:1050A00083F3118808BD8269936801339360D0E966
:1050B000003213605A60EDE7FFF7C0BF054BD968B7
:1050C00008751868026853601A600122D86002757A
:1050D000FBF7A0B9A06D00200C4B30B5DD684B1C70
:1050E00087B004460FD02B46094A684600F066F99F
:1050F0002046FFF7E3FF009B13B1684600F068F914
:10510000A86907B030BDFFF7D9FFF9E7A06D00200F
:105110007550000838B50C4D04468161EB68816814
:105120009A68914203D8BDE83840FFF787BF184618
:10513000FFF792FF01230146EC6020462375BDE88E
:105140003840FBF767B900BFA06D0020044B1A6818
:10515000DB6890689B68984294BF002001207047EC
:10516000A06D0020084B10B51C68D86822685360F9
:105170001A600122DC602275FFF76EFF01462046AF
:10518000BDE81040FBF746B9A06D002038B50123FB
:10519000084C00252370656000F0ACFD00F0D2FDE6
:1051A0000549064800F0A6FE0223237085F3118806
:1051B00038BD00BF08700020E0690008A06D002025
:1051C00008B572B6044B186500F0BEFB00F080FC19
:1051D000024B03221A70FEE7A06D00200870002029
:1051E00000F02CB98B600223086108468B8270475F
:1051F0008368A3F1840243F8142C026943F8442C19
:10520000426943F8402C094A43F8242CC268A3F1B0
:10521000200043F8182C022203F80C2C002203F87B
:105220000B2C034A43F8102C704700BF2D040008D4
:10523000A06D002008B5FFF7DBFFBDE80840FFF7D1
:105240003BBF0000024BDB6898610F20FFF736BFC1
:10525000A06D0020302383F31188FFF7F3BF000017
:1052600008B50146302383F311880820FFF734FF87
:10527000002383F3118808BD064BDB6839B142680F
:1052800018605A60136043600420FFF725BF4FF099
:10529000FF307047A06D00200368984206D01A685E
:1052A0000260506018469961FFF706BF7047000022
:1052B000036810B59C68A2420CD85C688A600B60D9
:1052C0004C602160596099688A1A9A604FF0FF33E8
:1052D000836010BD121B1B68ECE700000A2938BF71
:1052E0000A2170B504460D460A26601900F0FCFC40
:1052F00000F0E4FC041BA54203D8751C04462E46AE
:10530000F3E70A2E04D90120BDE8704000F032BE58
:1053100070BD0000F8B5144B0D460A2A4FF00A077D
:10532000D96103F11001826038BF0A224160196916
:105330001446016048601861A81800F0C5FC00F030
:10534000BDFC431B0646A34206D37C1C28192746F6
:10535000354600F0C9FCF2E70A2F04D90120BDE868
:10536000F84000F007BEF8BDA06D0020F8B5064675
:105370000D4600F0A3FC0F4A134653F8107F9F42DE
:1053800006D12A4601463046BDE8F840FFF7C2BFC5
:10539000D169BB68441A2C1928BF2C46A34202D9F4
:1053A0002946FFF79BFF224631460348BDE8F840F7
:1053B000FFF77EBFA06D0020B06D0020C0E9032381
:1053C000002310B45DF8044B4361FFF7CFBF00002A
:1053D00010B5194C236998420DD08168D0E900328C
:1053E00013605A609A680A449A60002303604FF081
:1053F000FF33A36110BD0268234643F8102F5360AA
:105400000022026022699A4203D1BDE8104000F0F8
:1054100065BC936881680B44936000F04FFC22697F
:10542000E1699268441AA242E4D91144BDE81040EF
:10543000091AFFF753BF00BFA06D00202DE9F04708
:10544000DFF8BC8008F110072C4ED8F8105000F09F
:1054500035FCD8F81C40AA68031B9A423ED8144475
:105460004FF00009D5E90032C8F81C4013605A60BB
:10547000C5F80090D8F81030B34201D100F02EFCEE
:1054800089F31188D5E9033128469847302383F3FF
:1054900011886B69002BD8D000F010FC6A69A0EB72
:1054A000040982464A450DD2022000F063FD002225
:1054B000D8F81030B34208D151462846BDE8F0472D
:1054C000FFF728BF121A2244F2E712EB0909294616
:1054D000384638BF4A46FFF7EBFEB5E7D8F810303C
:1054E000B34208D01444C8F81C00211AA960BDE8D2
:1054F000F047FFF7F3BEBDE8F08700BFB06D0020B6
:10550000A06D002038B500F0D9FB054AD2E9084566
:10551000031B181945F10001C2E9080138BD00BF9D
:10552000A06D002000207047FEE7000070470000DB
:105530004FF0FF3070470000BFF34F8F044B1A69E4
:105540005107FCD1D3F810215207F8D1704700BFA2
:105550000020005208B50D4B1B78ABB9FFF7ECFFEC
:105560000B4BDA68D10704D50A4A5A6002F1883237
:105570005A60D3F80C21D20706D5064AC3F8042195
:1055800002F18832C3F8042108BD00BF107000206A
:10559000002000522301674508B5114B1B78F3B971
:1055A000104B1A69510703D5DA6842F04002DA60FD
:1055B000D3F81021520705D5D3F80C2142F0400250
:1055C000C3F80C21FFF7B8FF064BDA6842F001027E
:1055D000DA60D3F80C2142F00102C3F80C2108BDB7
:1055E00010700020002000520F289ABF00F5806044
:1055F00040040020704700004FF400307047000066
:10560000102070470F2808B50BD8FFF7EDFF00F505
:1056100000330268013204D104308342F9D1012001
:1056200008BD0020FCE700000F2838B505463FD82C
:10563000FFF782FF1F4CFFF78DFF4FF0FF33072866
:105640006361C4F814311DD82361FFF775FF0302AD
:1056500043F02403E360E36843F08003E3602369DD
:105660005A07FCD42846FFF767FFFFF7BDFF4FF44A
:10567000003100F009FA2846FFF78EFFBDE83840F8
:10568000FFF7C0BFC4F81031FFF756FFA0F10803C1
:105690001B0243F02403C4F80C31D4F80C3143F05E
:1056A0008003C4F80C31D4F810315B07FBD4D9E780
:1056B000002038BD002000522DE9F84F05460C4669
:1056C000104645EA0203DE0602D00020BDE8F88F4E
:1056D00020F01F00DFF8BCB0DFF8BCA0FFF73AFFF6
:1056E00004EB0008444503D10120FFF755FFEDE727
:1056F00020222946204601F00BF810B9203520342D
:10570000F0E72B4605F120021F68791CDDD1043338
:105710009A42F9D105F178431B481C4EB3F5801F1E
:105720001B4B38BF184603F1F80332BFD946D146A8
:105730001E46FFF701FF0760A5EB040C336804F178
:105740001C0143F002033360231FD9F8007017F0E7
:105750000507FAD153F8042F8B424CF80320F4D1FB
:10576000BFF34F8FFFF7E8FE4FF0FF3320222146B3
:1057700003602846336823F00203336000F0C8FF5B
:105780000028BBD03846B0E7142100520C2000524C
:1057900014200052102000521021005210B5084C65
:1057A000237828B11BB9FFF7D5FE0123237010BD64
:1057B000002BFCD02070BDE81040FFF7EDBE00BF0D
:1057C000107000202DE9F04F0D4685B0814658B18C
:1057D00011F00D0614BF2022082211F008030193D6
:1057E00004D0431E03426AD0002435E0002E37D097
:1057F00009F11F0121F01F094FF00108324F05F098
:105800000403DFF8D0A005EA080BBBF1000F32D08B
:105810007869C0072FD408F101080C37B8F1060FDA
:10582000F3D19EB9294D4946A819019200F0ACFA6E
:10583000044600283AD11836019A782EF3D1494609
:1058400000F0A2FA0446002830D1019A49462048C7
:1058500000F09AFA044668BB204605B0BDE8F08F18
:105860000029C9D101462846029200F08DFA04466B
:10587000E0B9029AC0E713B178694107CBD5AC070C
:1058800002D578698007C6D5019911B178690107F9
:10589000C1D51820494600FB08A0CDE9022300F03D
:1058A00073FA0446DDE902230028B4D04A460021F9
:1058B000204601E04A460021FCF796F8CCE7024674
:1058C000002E95D198E700BFEC69000844700020D5
:1058D000147000202C7000200121FFF773BF00001E
:1058E000F8B5144D01241827134E40F2FF32002161
:1058F0000120FCF779F807FB046001342A6955F8A8
:105900000C1F00F02DFA062CF5D137254FF4C054AA
:105910002046FFF7E1FF014628B122460748BDE8CF
:10592000F84000F01DBAC4EBC404013D4FEAD404B2
:10593000EED1F8BDEC6900082C7000201470002036
:1059400008B100F093BA704738B5054D0024033410
:10595000696855F80C0B00F0A9F8122CF7D138BD86
:10596000EC69000838B5EFF311859DB9EFF30584B4
:10597000C4F30804302334B183F31188FFF7C2FD68
:1059800085F3118838BD83F31188FFF7BBFD84F3DD
:10599000118838BDBDE83840FFF7B4BD10B5FFF73A
:1059A000E1FF104CC008104A002340EA4170C908CA
:1059B000A0FB04ECA0FB020E1CEB0000A1FB044CBE
:1059C000A1FB02125B41001943EB0C0011EB0E012D
:1059D00042F10002411842F10000090941EA007059
:1059E00010BD00BFCFF753E3A59BC4200244074B73
:1059F000D2B210B5904200D110BD441C00B253F891
:105A0000200041F8040BE0B2F4E700BF504000581A
:105A10000E4B30B51C6F240405D41C6F1C671C6F23
:105A200044F400441C670A4C02442368D2B243F495
:105A300080732360074B904200D130BD441C51F865
:105A4000045B00B243F82050E0B2F4E7004402588F
:105A5000004802585040005807B5012201A9002013
:105A6000FFF7C4FF019803B05DF804FB13B50446CB
:105A7000FFF7F2FFA04205D0012201A90020019406
:105A8000FFF7C6FF02B010BD0144BFF34F8F064BB6
:105A9000884204D3BFF34F8FBFF36F8F7047C3F8B3
:105AA0005C022030F4E700BF00ED00E00144BFF3EA
:105AB0004F8F064B884204D3BFF34F8FBFF36F8FD6
:105AC0007047C3F870022030F4E700BF00ED00E03B
:105AD00070470000114BDA6952021ED59A69D0074F
:105AE00004D50F4A9A6002F144329A600B4BDA698E
:105AF000D107FCD41A6A22F480021A629A6942F031
:105B000002029A61DA69D207FCD49A6942F0010272
:105B10009A61024AD369DB07FCD470470020005227
:105B20003B2A1908074B45F255521A6003225A6066
:105B300040F2FF729A604CF6CC421A600122024B8E
:105B40001A70704700480058C0700020034B1B7843
:105B50001BB1034B4AF6AA221A607047C07000209E
:105B600000480058034B1A681AB9034AD2F8D024E7
:105B70001A607047BC70002000400258024B4FF47E
:105B80008032C3F8D02470470040025808B5FFF7B0
:105B9000E9FF024B1868C0F3806008BDBC700020AC
:105BA00070B5BFF34F8FBFF36F8F1A4A0021C2F851
:105BB0005012BFF34F8FBFF36F8F536943F400331D
:105BC0005361BFF34F8FBFF36F8FC2F88410BFF3E1
:105BD0004F8FD2F8803043F6E074C3F3C900C3F3AB
:105BE0004E335B0103EA0406014646EA817501393A
:105BF000C2F86052F9D2203B13F1200FF2D1BFF36B
:105C00004F8F536943F480335361BFF34F8FBFF31A
:105C10006F8F70BD00ED00E0FEE70000214B2248D1
:105C2000224A70B5904237D3214BC11EDA1C121A9A
:105C300022F003028B4238BF00220021FBF7D4FE82
:105C40001C4A0023C2F88430BFF34F8FD2F8803053
:105C500043F6E074C3F3C900C3F34E335B0103EAB8
:105C60000406014646EA81750139C2F86C52F9D240
:105C7000203B13F1200FF2D1BFF34F8FBFF36F8F93
:105C8000BFF34F8FBFF36F8F0023C2F85032BFF3C3
:105C90004F8FBFF36F8F70BD53F8041B40F8041B88
:105CA000C0E700BFB46B0008E4700020E47000207F
:105CB000E470002000ED00E000F05ABA014B586A91
:105CC000704700BF000C0040034B002258631A616C
:105CD0000222DA60704700BF000C0040014B002236
:105CE000DA607047000C0040014B5863704700BFFA
:105CF000000C0040024B034A1A60034A5A60704786
:105D0000C4700020E870002000000220074B4942C8
:105D100010B55C68201A08401968821A8A4203D3B9
:105D2000A24201D85A6010BD0020FCE7C4700020D8
:105D300008B5302383F31188FFF7E8FF002383F3CE
:105D4000118808BD04480121044B03600023C0E909
:105D500001330C3000F016B9CC700020315D000822
:105D6000CB1D083A23F00703591A521A012110B427
:105D7000D2080024C0E9004384600C301C605A60E3
:105D80005DF8044B00F0FEB82DE9F84F364ECD1DFE
:105D90000F46002818BF0646082A4FEAD50538BF27
:105DA000082206F10C08341D9146404600F006F921
:105DB00009F10701C9F1000E224624686CB940467A
:105DC00000F006F93368CBB308224946E80098474B
:105DD000044698B340E9026730E004EB010CD4F8C4
:105DE00004A00CEA0E0C0AF10100ACF1080304EB6C
:105DF000C0009842E0D9A0EB0C0CB5EBEC0F4FEAD9
:105E0000EC0BD9D89C421CD204F10802AB45A3EBA1
:105E100002024FEAE202626009D9691CED43206880
:105E200003EBC1025D44556043F8310022601C461B
:105E30005F60404644F8086B00F0CAF82046BDE8B1
:105E4000F88FAA45216802D111602346EFE701359A
:105E500004EBC50344F8351003F10801401AC010E3
:105E600058601360F1E700BFCC700020F8B550F81F
:105E7000043C044650F8085CA0F1080607332F1DC7
:105E80000C35DB0840F8043C284600F097F83B4608
:105E90009F421A6801D0B34228D20AB1964225D255
:105EA00044F8082C54F8042C1E60013254F8081CE5
:105EB00006EBC200814206D14868024444F8042C33
:105EC0000A6844F8082C5868411C03EBC1018E4253
:105ED00007D154F8042C013202445A6054F8082CBB
:105EE0001A602846BDE8F84000F072B81346CFE7C4
:105EF000FEE7000070B51B4B0025044686B05860D5
:105F00000E4685620163FEF771FA04F11003A56085
:105F1000E562C4E904334FF0FF33C4E90044C4E947
:105F20000635FFF7CBFE2B46024604F1340120462E
:105F3000C4E9082380230C4A2565FFF753F90123A0
:105F40000A4AE06000920375684672680192B2687E
:105F5000CDE90223064BCDE90435FFF76BF906B016
:105F600070BD00BF08700020346A0008396A00085C
:105F7000F15E0008024AD36A1843D062704700BF3E
:105F8000A06D0020C0E90000816070478368013B7C
:105F9000002B10B583600CDA074BDC684368A06106
:105FA000206063601C6044600520FFF787F8A069EB
:105FB00010BD0020FCE700BFA06D002008B5302315
:105FC00083F31188FFF7E2FF002383F3118808BDF4
:105FD00008B5302383F3118883680133002B836075
:105FE00007DC036800211A68026050601846FFF75A
:105FF00091F8002383F3118808BD00004B684360CB
:106000008B688360CB68C3600B6943614B69036233
:106010008B6943620B6803607047000008B53C4B16
:1060200040F2FF713B48D3F888200A43C3F8882028
:10603000D3F8882022F4FF6222F00702C3F88820F8
:10604000D3F88830344B1A6C0A431A649A6E0A43A8
:106050009A66324A9B6E1146FFF7D0FF00F58060CA
:1060600002F11C01FFF7CAFF00F5806002F1380160
:10607000FFF7C4FF00F5806002F15401FFF7BEFF97
:1060800000F5806002F17001FFF7B8FF00F5806055
:1060900002F18C01FFF7B2FF00F5806002F1A80168
:1060A000FFF7ACFF00F5806002F1C401FFF7A6FF27
:1060B00000F5806002F1E001FFF7A0FF00F58060CD
:1060C00002F1FC01FFF79AFF02F58C7100F5806088
:1060D000FFF794FF00F00EF9114BD3F8902242F035
:1060E0000102C3F89022D3F8942242F00102C3F8CF
:1060F00094220522C3F898204FF06052C3F89C20E8
:10610000084AC3F8A020BDE80840FFF7E3BC00BF81
:10611000004402580000025800450258406A000836
:1061200000ED00E01F00080308B500F0CFFAFFF70C
:106130002DF80C4BDA6B42F04002DA635A6E22F013
:1061400040025A665B6E084B1A6842F008021A60F9
:106150001A6842F004021A60FFF704FDBDE8084027
:10616000FFF7BEBB00450258001802487047000008
:106170000E4B9A6C42F008029A641A6F42F00802C1
:106180001A670B4A1B6FD36B43F00803D363C72214
:10619000084B9A624FF0FF32DA6200229A615A632A
:1061A000DA605A6001225A611A607047004502584D
:1061B0000010005C000C0040094A08B51169D36862
:1061C0000B40D9B29B076FEA0101116107D530235B
:1061D00083F31188FFF704F8002383F3118808BDC7
:1061E000000C0040044BDA6B0243DA635A6E104332
:1061F00058665B6E704700BF0045025808B53C4BBF
:106200004FF0FF31D3F8802062F00042C3F88020C5
:10621000D3F8802002F00042C3F88020D3F8802019
:10622000D3F88420C3F88410D3F884200022C3F864
:106230008420D3F88400D86F40F0FF4040F4FF0082
:1062400040F4DF4040F07F00D867D86F20F0FF4077
:1062500020F4FF0020F4DF4020F07F00D867D86FE3
:10626000D3F888006FEA40506FEA5050C3F88800B6
:10627000D3F88800C0F30A00C3F88800D3F8880078
:10628000D3F89000C3F89010D3F89000C3F8902092
:10629000D3F89000D3F89400C3F89410D3F8940086
:1062A000C3F89420D3F89400D3F89800C3F898105A
:1062B000D3F89800C3F89820D3F89800D3F88C004E
:1062C000C3F88C10D3F88C00C3F88C20D3F88C0062
:1062D000D3F89C00C3F89C10D3F89C10C3F89C2002
:1062E000D3F89C30FEF72CFABDE8084000F0BEB9A8
:1062F0000044025808B50122504BC3F80821504B06
:106300005A6D42F002025A65DA6F42F00202DA6711
:106310000422DB6F4B4BDA605A689104FCD54A4A81
:106320001A6001229A60494ADA6000221A614FF429
:1063300040429A61434B9A699204FCD51A6842F430
:1063400080721A60424B1A6F12F4407F04D04FF4EF
:1063500080321A6700221A671A6842F001021A6036
:106360003B4B1A685007FCD500221A611A6912F0DB
:106370003802FBD1012119604FF0804159605A6702
:10638000344ADA62344A1A611A6842F480321A6076
:106390002F4B1A689103FCD51A6842F480521A6098
:1063A0001A689204FCD52D4A2D499A6200225A633C
:1063B000196301F57C01DA6301F5E77199635A64A9
:1063C000284A1A64284ADA621A6842F0A8521A6007
:1063D0001F4B1A6802F02852B2F1285FF9D1482207
:1063E0009A614FF48862DA6140221A621F4ADA64C5
:1063F0001F4A1A651F4A5A651F4A9A6532231F4A67
:106400001360136803F00F03022BFAD1104A1369CB
:1064100043F003031361136903F03803182BFAD117
:106420004FF00050FFF7DEFE4FF08040FFF7DAFE3E
:106430004FF00040BDE80840FFF7D4BE0080005197
:10644000004502580048025800C000F00400000156
:10645000004402580000FF010088900832206000CC
:1064600063020901470E0508DD0BBF012000002073
:10647000000001100910E00000010110002000528E
:106480004FF0B04208B5D2F8883003F00103C2F8EB
:10649000883023B1044A13680BB150689847BDE8AF
:1064A0000840FDF7CBBF00BF486400204FF0B0426A
:1064B00008B5D2F8883003F00203C2F8883023B15F
:1064C000044A93680BB1D0689847BDE80840FDF7CF
:1064D000B5BF00BF486400204FF0B04208B5D2F805
:1064E000883003F00403C2F8883023B1044A1369EA
:1064F0000BB150699847BDE80840FDF79FBF00BF4A
:10650000486400204FF0B04208B5D2F8883003F05C
:106510000803C2F8883023B1044A93690BB1D069EB
:106520009847BDE80840FDF789BF00BF48640020D8
:106530004FF0B04208B5D2F8883003F01003C2F82B
:10654000883023B1044A136A0BB1506A9847BDE8FA
:106550000840FDF773BF00BF486400204FF0B04310
:1065600010B5D3F8884004F47872C3F88820A306E5
:1065700004D5124A936A0BB1D06A9847600604D5D5
:106580000E4A136B0BB1506B9847210604D50B4A8A
:10659000936B0BB1D06B9847E20504D5074A136C97
:1065A0000BB1506C9847A30504D5044A936C0BB10A
:1065B000D06C9847BDE81040FDF740BF486400200C
:1065C0004FF0B04310B5D3F8884004F47C42C3F8D0
:1065D0008820620504D5164A136D0BB1506D98479B
:1065E000230504D5124A936D0BB1D06D9847E00492
:1065F00004D50F4A136E0BB1506E9847A10404D511
:106600000B4A936E0BB1D06E9847620404D5084ACA
:10661000136F0BB1506F9847230404D5044A936F4E
:106620000BB1D06F9847BDE81040FDF707BF00BF22
:106630004864002008B50348FEF788FABDE8084022
:10664000FDF7FCBEC864002008B50348FEF77EFADB
:10665000BDE80840FDF7F2BE3465002008B5FFF73D
:10666000ABFDBDE80840FDF7E9BE0000062108B516
:106670000846FEF7F1FA06210720FEF7EDFA06219B
:106680000820FEF7E9FA06210920FEF7E5FA0621BF
:106690000A20FEF7E1FA06211720FEF7DDFA0621AF
:1066A0002820FEF7D9FA09217A20FEF7D5FA07212A
:1066B0003220FEF7D1FA0C212520FEF7CDFA0C216D
:1066C0005320BDE80840FEF7C7BA000008B5FFF741
:1066D00095FDFEF7FDF8FEF77DFCFFF747FDBDE8F1
:1066E0000840FFF7E9BA00000B460146184600F0E3
:1066F00001B8000010B5054C13462CB10A460146FE
:106700000220AFF3008010BD2046FCE7000000002F
:1067100010B501390244904201D1002005E0037810
:1067200011F8014FA34201D0181B10BD0130F2E750
:106730002DE9F041A3B1C91A17780144044603F1C9
:10674000FF3C8C42204601D9002009E00578BD427B
:1067500004F10104F5D10CEB0405D618A54201D1D2
:10676000BDE8F08115F8018D16F801EDF045F5D082
:10677000E7E70000034611F8012B03F8012B002A7C
:10678000F9D17047636F6D2E6375626570696C6FC8
:10679000742E6865726534666300000053544D338F
:1067A0003248373F3F3F0053544D333248373378F8
:1067B0002F3732780053544D3332483734332F3724
:1067C00035332F373530000001105A0003105900BF
:1067D000012058000320560040A2E4F164689106AD
:1067E0000041A3E5F26569920700000043414E466F
:1067F0004449666163653A204D657373616765203E
:1068000052414D204F766572666C6F772100000013
:106810004261642043414E496661636520696E644C
:1068200065782E00000100000001FF0000A000407C
:1068300000A400400000000000000000092B000838
:106840009123000891320008012400080D2400085B
:106850002528000885250008C9230008CD23000845
:10686000A52300088D230008E1270008B1230008B4
:10687000F9330008BD230008B527000801040E0500
:10688000054B02020E05054B04010E05054B0501E3
:106890000B04044B080106030346000010000240ED
:1068A000080002400008024000000B0028000240DF
:1068B000080002400408024006010C0040000240AB
:1068C000080002400808024010020D005800024073
:1068D000080002400C08024016030E00700002403F
:1068E0000C0002401008024000040F008800024023
:1068F0000C0002401408024006051000A0000240EF
:106900000C0002401808024010061100B8000240B6
:106910000C0002401C08024016072F001004024021
:106920000804024020080240000838002804024001
:1069300008040240240802400609390040040240CD
:106940000804024028080240100A3A005804024095
:10695000080402402C080240160B3B007004024061
:106960000C04024030080240000C3C008804024045
:106970000C04024034080240060D4400A00402400A
:106980000C04024038080240100E4500B8040240D2
:106990000C0402403C080240160F4600009600001E
:1069A00000000000000000000000000000000000E7
:1069B0000000000000000000954F0008814F000813
:1069C000BD4F0008A94F0008B54F0008A14F0008AF
:1069D0008D4F0008794F0008C94F00086330000050
:1069E000DC690008F86D002008700020000100201C
:1069F00000FF010002000000000000300000040061
:106A0000080000000000002400000800040000004E
:106A10000004000000FC0000020000000000043040
:106A200000800000080000000000003800000100A5
:106A3000010000006D61696E0069646C6500000012
:106A40000000002800000000AAAAAAAA0000002452
:106A5000FFFF0000000000000000000000A0550A39
:106A600000000000AAAA9AAA00500000FFF200004D
:106A70000000007700009900000000000000000006
:106A8000AAAAAAAA00000000FFFF00000000000060
:106A9000000000005A000000000000009AAAAAAA04
:106AA00000000000F3FF000099000000000000005B
:106AB0000A00000000000000AAAAAAAA050000001F
:106AC000FFFF000088000000000000000000000040
:106AD00000000000AAAAAAAA00000000FFFF000010
:106AE00000000000000000000000000000000000A6
:106AF000AAAAAAAA00000000FFFF000000000000F0
:106B0000000000000000000000000000AAAAAAAADD
:106B100000000000FFFF0000000000000000000077
:106B20000000000000000000AAAAAAAA00000000BD
:106B3000FFFF000000000000000000000000000057
:106B400000000000AAAAAAAA00000000FFFF00009F
:106B50000000000000000000000000000000000035
:106B6000AAAAAAAA00000000FFFF0000000000007F
:106B700000000000000000001304000000000000FE
:106B80000000180000000000FE2A0100D2040000EE
:106B9000FF000000C86400203465002000000000F1
:106BA0009C67000883040000A767000850040000E9
:046BB000B5670008BD
:00000001FF
